:020000040800F2
:1000000000800020BDBF0008DFC00008E1C000087C
:1000100000000000000000000000000000000000E0
:10002000000000000000000000000000E3C0000825
:100030000000000000000000E5C000082D9300084B
:10004000F1BF0008F3BF0008F5BF0008F7BF0008C4
:10005000F9BF0008FBBF0008FDBF0008D5960008E7
:1000600001C000087193000805C0000807C000081F
:1000700009C000080BC000080DC000080FC0000830
:1000800011C0000813C0000815C0000817C0000800
:1000900019C00008019700081DC000081FC0000813
:1000A00021C0000823C0000825C000085D94000896
:1000B00029C000082BC000082DC000082FC0000870
:1000C000EDAF16204A62304029BD56B31544E9BF52
:1000D00077900D9CFE0B88C07E2615FA83807340B6
:0800E0000FCE674B80D541C033
:1000E800000000000000244000000000000059400B
:1000F800000000000088C3400000000084D797413A
:100108000080E03779C34143176E05B5B5B893460B
:10011800F5F93FE9034F384D321D30F94877825AD7
:080128003CBF737FDD4F15752C
:1001300001000000000000000A00000000000000B4
:100140006400000000000000E80300000000000060
:100150001027000000000000A08601000000000041
:1001600040420F0000000000809698000000000050
:1001700000E1F5050000000000CA9A3B0000000005
:1001800000E40B540200000000E87648170000006D
:100190000010A5D4E800000000A0724E180900006D
:1001A00000407A10F35A00000080C6A47E8D030040
:1001B0000000C16FF286230000008A5D784563016C
:1001C000000064A7B3B6E00D0000E8890423C78AE5
:1001D00010B5816A8A6D50231A428A6D05D0D20605
:1001E00002D4096D496B884710BD012043021A43B0
:1001F0008A650A68D3681B059B0F02D01049086006
:1002000010BD8B7E002BF9D113681B07F6D59368C0
:100210005B0709D4583153680C24A3435360FF2370
:1002200002330A689A4305E08A6D202313438B65E5
:10023000CA6D5C3102430A600149086010BDC046C6
:04024000080F002083
:10024400F0B58BB000240A9454259A4E715D0129AF
:1002540000D111E10127775531688A68520714D417
:10026400336942680992022A944A13D104273B4312
:1002740093426AD1904AD3430268D04318438B6AAD
:1002840003408B62002A64D4F5E0B06D2021014361
:10029400B165F0E0089104210B439342864B67D18A
:1002A40007683B4008998A6A1A438A623A024B6992
:1002B400934380681040824A02401A434A61002FE7
:1002C40000D4D8E001237F483A4607680720800518
:1002D4003946099001407C480792824200D08EE062
:1002E400D8053A46024000D089E0764F3A68099B27
:1002F4009A431143014339607648006876490AF00D
:1003040083FB0C2141430C310A910A98002800D147
:10031400B1E00A98401E0A900A98002800D1AAE089
:100324000A98401E0A900A98002800D1A3E00A986F
:10033400401E0A900A98002800D19CE00A98401EAA
:100344000A900A980028E4D195E00268002A00D4B3
:1003540091E05C4801685D4B9A4200D182E05C4BBD
:100364009A427CD0584B9A4200D084E005227AE02D
:10037400029106941F26099A16400F2201920596AF
:10038400B2404C4E346E03929443049402681A4271
:10039400079249D0D207069C2346089948D1079A68
:1003A40092073B4644D4079B5A0767D41A0767D47D
:1003B400DA06029B3CD4079B9A0663D45A0663D49C
:1003C4001A0663D4DA0563D49A0563D45A0563D450
:1003D4001A0563D4DA0463D49A0463D45A0463D444
:1003E4001A04019B24D4079AD2035FD4079A920378
:1003F4005ED4079A5203D2171223134018E03348ED
:10040400079A824202D11806814205D330488242BB
:1004140031D1980507402ED12A4F3A68099B9A4357
:1004240011430143396026E05200D30E069C08991B
:10043400059FBB40049A13433366099A9208F369F3
:1004440093420AD9039AD2438B6A13403E46079FCC
:10045400BA00120FB240174E26E7079F26E7032281
:10046400D20501E003229205114007229205036898
:1004740093435918016074550BB0F0BD0223D7E7BC
:100484000323D5E70523D3E70623D1E70723CFE7E3
:100494000823CDE70923CBE70A23C9E70B23C7E7E2
:1004A4000C23C5E70D23C3E70E23C1E71023BFE7E1
:1004B4001123BDE7840D0020FFFF07000400008026
:1004C40000FFFF0708270140001000B0004000B8FB
:0C04D400002000B420000020400D0300B8
:1004E000F0B5684B02225A771A68956801242543B3
:1004F00095601D6A012D43D0022D0DD0032D00D033
:100500008AE00D40042900D389E00021002D00D0AD
:1005100091E010685C77F0BD4D0813D06E1E032E7D
:1005200018D2032635400BD0468807883F04BE19F1
:100530001660012D04D0C5888688360475191560AB
:100540000D46A543C907E4D06900405A10801068E1
:100550005C77F0BD418803881B0459181160C1887D
:1005600083881B0459181160418903891B04591899
:100570001160C18983891B04591811601030E9E7A3
:100580008D0811D06D1E032D18D20E070425B60F4D
:100590000AD00678360647783F04BE1987783F02AE
:1005A000F619C778F61916600326314003295DD085
:1005B000022951D0012961D1405D5EE00178090630
:1005C00043781B04591883781B02C918C378C918CB
:1005D00011600179090643791B04591883791B02BC
:1005E000C918C379C9181160017A0906437A1B0436
:1005F0005918837A1B02C918C37AC9181160017B84
:100600000906437B1B045918837B1B02C918C37B53
:10061000C91811601030D1E700205C77F0BD016887
:1006200011604168116081681160C1681160042126
:10063000002D00D16DE7890046581660012D00D1CC
:1006400067E7401841681160022D00D161E78068BA
:10065000106010685C77F0BD41194978405D000278
:10066000401810801A6810685C77F0BD4119405D31
:1006700000024D7840191080887810701A68106850
:080680005C77F0BDBC0E002008
:10068800F0B585B0634C2178002902D0022005B06E
:10069800F0BD029203930490012626705E4A116809
:1006A80037045E4C2068C0032BD420685C4B5D1C6B
:1006B800019525601842304600D0A6E00120009040
:1006C8008604206840033CD4606800990843606051
:1006D800049802990160BFF36F8F03994160116814
:1006E800206838424DD12068019B23604C4B18424A
:1006F800009800D085E020680023304261D10020B6
:100708007FE07D20C5001068431A0320AB427CD2ED
:1007180023683B42C9D013685B1AAB4275D2236881
:100728003B42C2D013685B1AAB426ED223683B428D
:10073800BBD013685B1AAB4267D220683842E2D15B
:10074800B3E77D20C5001068431A0320AB425CD292
:1007580023683342B8D013685B1AAB4255D223687A
:100768003342B1D013685B1AAB424ED2236833428E
:10077800AAD013685B1AAB4247D220683042E2D154
:10078800A2E77D20C3001068451A03209D4238D295
:1007980025683D42A7D015686D1A9D4231D225685B
:1007A8003D42A0D015686D1A9D422AD225683D4267
:1007B80099D015686D1A9D4223D220683842E2D13B
:1007C80091E77D20C5001068471A0320AF4218D270
:1007D8002768374214D017687F1AAF4211D22768AA
:1007E80037420DD017687F1AAF420AD227683742BE
:1007F80006D017687F1AAF4203D220683042E2D190
:1008080018466168009A914361600021014A11709D
:1008180005B0F0BD880F0020240000201020024001
:04082800FA8300004F
:10082C0070B52B490B6801222A480468E4030ED4E6
:10083C000468294D6E1C06602C4202D104686403C6
:10084C0025D4D10742680A434260406870BD140445
:10085C007D25ED000E68F61AAE42F2D206682642ED
:10086C00E6D00E68F61AAE42EBD206682642DFD00E
:10087C000E68F61AAE42E4D206682642D8D00E684C
:10088C00F61AAE42DDD206682642E3D1D0E79404D4
:10089C007D25ED000E68F61AAE42D2D206682642CD
:1008AC00CFD00E68F61AAE42CBD206682642C8D01C
:1008BC000E68F61AAE42C4D206682642C1D00E6843
:1008CC00F61AAE42BDD206682642E3D1B9E7C0465D
:0C08DC002400002010200240FA830000DD
:1008E80070B52B490B6801222A480468E4030ED42A
:1008F8000468294D6E1C06602C4202D1046864030A
:1009080025D4910742680A434260406870BD1404C8
:100918007D25ED000E68F61AAE42F2D20668264230
:10092800E6D00E68F61AAE42EBD206682642DFD051
:100938000E68F61AAE42E4D206682642D8D00E688F
:10094800F61AAE42DDD206682642E3D1D0E7940417
:100958007D25ED000E68F61AAE42D2D20668264210
:10096800CFD00E68F61AAE42CBD206682642C8D05F
:100978000E68F61AAE42C4D206682642C1D00E6886
:10098800F61AAE42BDD206682642E3D1B9E7C046A0
:0C0998002400002010200240FA83000020
:1009A400F0B586B06B490A78002A02D0022006B05E
:1009B400F0BD059001200870674C22680504674B60
:1009C4001968C90320D41968654E771C04971F6001
:1009D4003142014600D0B5E0012001908604186838
:1009E400400334D40022D043059908605D48007860
:1009F4005D49096808180290814200D398E000928A
:100A04007D20C200594F48E07D21CE0021688F1A15
:100A14000321B74200D395E01F682F42D3D0276843
:100A2400BF1AB74200D38DE01F682F42CBD027688E
:100A3400BF1AB74200D385E01F682F42C3D027688E
:100A4400BF1AB7427ED219682942DFD1BBE77D20A5
:100A5400C00021688F1A0321874273D21F6837426E
:100A6400C0D02768BF1A87426CD21F683742B9D0FA
:100A74002768BF1A874265D21F683742B2D02768F9
:100A8400BF1A87425ED219683142E2D1AAE70399BC
:100A9400491C02988142354F5AD058683840039116
:100AA400C9000143A81C08435860206819682942FA
:100AB4001AD021680F1A032197423CD21F682F4293
:100AC40012D027683F1A974235D21F682F420BD0A5
:100AD40027683F1A97422ED21F682F4204D02768F6
:100AE4003F1A9742E2D326E01968049F1F601C4F07
:100AF40039421FD119683142C9D021680F1A032124
:100B0400974218D21F683742C1D027683F1A9742CC
:100B140011D21F683742BAD027683F1A97420AD2C7
:100B24001F683742B3D027683F1A9742E2D302E0E6
:100B3400002103E001990598039A02605868022293
:100B4400904358600020034A1070084606B0F0BD78
:100B54000099F3E7880F00202400002010200240B1
:100B6400FA8300008C0F00205C0F002005E0FEFFDC
:100B7400F0B583B0814A1178002902D0022003B075
:100B8400F0BD012414700168CA077D4A0BD0416886
:100B9400012901D0202100E01C218368C5682D04AF
:100BA4001D435550016806230B40062B0BD101460B
:100BB40010312AC90D43FF208343C14359401069B2
:100BC4000840284323E08B070DD4490720D5416909
:100BD400FF239943DB434B4015691169EDB2AA2DFC
:100BE4000DD12E460CE01169664B0B40FF21C94321
:100BF400594015690D4000692843184307E0BB2696
:100C04001940CC2D00D1CC268069304308431061B3
:100C14005D4B196825041068C00326D410685B4E28
:100C2400771C029717603042204600D0A1E00120D3
:100C3400019084041068400337D40198410450683B
:100C44000091084350601968106828424DD110681B
:100C5400029D15604D4D2842019800D085E0106832
:100C64000025204261D100207FE07D20C600186865
:100C7400471A0320B7427CD217682F42CED01F6890
:100C84007F1AB74275D217682F42C7D01F687F1AE0
:100C9400B7426ED217682F42C0D01F687F1AB7427E
:100CA40067D210682842E2D1B8E77D20C7001868EF
:100CB400461A0320BE425CD216682642BDD01E6886
:100CC400761ABE4255D216682642B6D01E68761AE7
:100CD400BE424ED216682642AFD01E68761ABE4275
:100CE40047D210682042E2D1A7E77D20C7001868E8
:100CF400461A0320BE4238D216682E42A7D01E6878
:100D0400761ABE4231D216682E42A0D01E68761AD8
:100D1400BE422AD216682E4299D01E68761ABE4266
:100D240023D210682842E2D191E77D20C6001868DA
:100D3400471A0320B74218D21768274214D01F68F5
:100D44007F1AB74211D2176827420DD01F687F1A45
:100D5400B7420AD21768274206D01F687F1AB742E3
:100D640003D210682042E2D128465168009B99437F
:100D740051600021014A117003B0F0BD880F0020BA
:100D84001020024000604F0724000020FA83000076
:100D9400F0B58CB00F460968002900D1BCE00646C6
:100DA4005E48864201D0052000E003200090012423
:100DB40000250A950B950394029701960FE01943B9
:100DC400116039680846E040AD1C0A9A121D0A9267
:100DD4000B9A08320B92641C002800D19CE0601E20
:100DE400039B0990834019400791EAD004943E463E
:100DF40003273846A840C0432C4675682946394025
:100E04004A1E012A0695059413D808900198826811
:100E1400089F3A40F7680646A74017438760EA06EA
:100E2400D20F09988240089877689F4317437760E8
:100E340007E00329019E04D1029F2B462546049C0A
:100E44001FE0F2680240029FBB682546A34013439B
:100E5400F3600229069B049C13D108901C200A9974
:100E640008400F218140099AD2089200B218136AEF
:100E74008B43396981400898194311627B680321C7
:100E84001940A940326802400A4332609803800F37
:100E940097D0032009998143214840180521090767
:100EA4008E42016E0AD0204A964205D01F4A9642CD
:100EB400009B04D1022302E0012300E00023182256
:100EC4000B9E32400F269640B143603093400B4353
:100ED4000360134801687868C20202D5079B19436E
:100EE40001E0079B99430E4A11605168820201D5C3
:100EF400194300E099430A4A51600A494968820348
:100F040001D5194300E09943064A51601168C003B2
:100F140000D554E7994353E70CB0F0BD000C0050E2
:100F240000180240801802400004005000080050DD
:100F3400F0B585B003AD00242C70384F3E689B1B80
:100F44009E18374A1268232353431A0D72433D46B1
:100F54003F680492029003689A680A421AD00322F6
:100F640001925202914218D10094284602E09968F5
:100F740011424DD0197B03AC217003990168C91B40
:100F8400B1421DD20499049C641E04940029EED13C
:100F94000026ECE7002005B0F0BD284603E09A687F
:100FA4000A422C4637D00268D21BB24208D22546E8
:100FB400049A049C641E0494002AF0D10026EEE7EF
:100FC4005968E0229143596041218900029842689E
:100FD4008A420BD181680122D403A14202D0920239
:100FE400914203D1196840229143196001214A03B7
:100FF400846A5C30944205D11C6894431C601C686C
:1010040014431C60002202704170019805B0F0BDC9
:10101400009805B0F0BD204605B0F0BD24000020C6
:041024002000002088
:10102800F0B582B0254C2368D21A551824490968AE
:101038004901090D694326680191026893680021F6
:101048001B0637D503465C33009302E093681B0602
:1010580030D52768BF1BAF4207D2019F019B5B1E9B
:101068000193002FF2D10025F0E75168E024A14355
:1010780051604121890044688C420BD18168012468
:10108800E503A94202D0A402A14203D11168402479
:10109800A143116001214C03806AA04205D1106868
:1010A800A04310601068204310600020009A107060
:1010B80051700321084602B0F0BDC046240000204C
:0410C80020000020E4
:1010CC00F0B589B05C249C4E335D012B00D131E12D
:1010DC00012705943755994B1B6806935D230493A0
:1010EC00F35C012B6FD1002800D120E1002900D145
:1010FC001DE1049BF35C042B02D00523049C3355A7
:10110C000390002333664625725344243253F287EE
:10111C00F4688B48029484423C4600D30024240398
:10112C000194380337687C6884430020019BE418E1
:10113C007C603164039BB363F0643065B2873A68BA
:10114C00520603D43A68402313433B60029A7C4B0B
:10115C009A427268069C43D3002A039806D10288EF
:10116C00FA60801CB063F28F521EF287012205E0F8
:10117C00724B1B681B1B0A2B00D3D5E0F38F002B83
:10118C0002D1735B002B6AD0BB689B070CD5F38F25
:10119C00002B09D0012A07D10288FA60801CB063A9
:1011AC00F28F521EF2870022BB68DB07E0D0735B24
:1011BC00002BDDD0FA680A80725B521E7253891CB8
:1011CC0031640122D4E74124A4007568A54200D003
:1011DC00ADE0042B00D0AAE0B368002B83D0A6E0CE
:1011EC00002A039807D100783873B06B401CB063A9
:1011FC00F08F401EF087012005E050490968091B5B
:10120C000A2900D390E0F18F002901D0376803E060
:10121C00715B0029376822D0B96889070ED5F18F28
:10122C0000290BD0012809D1B06B00783873B06B52
:10123C00401CB063F08F401EF0870020B968C907CE
:10124C00DBD0715B0029D8D0387B316C0870705BB7
:10125C00401E7053306C401C30640120CDE707A851
:10126C000021039101703748006823214143090D87
:10127C00324A1068201A0A3041431268089103253B
:10128C00B968C904890F12D0EB0203E0B96819429E
:10129C00069C0CD029490968891A814217D20899F1
:1012AC00089C641E08940029F0D10020EEE7224827
:1012BC000A212246FFF7B2FE00282DD169021E48F2
:1012CC000A222346FFF730FE002825D129E0786852
:1012DC00E0218843786041208000716881420BD105
:1012EC00B1680120C203914202D08002814203D135
:1012FC00386840218843386001214A03B06A904223
:10130C00059B05D1386890433860386810433860C5
:10131C000398F05404983154306E20210843306601
:10132C003166306E002802D10120049970540020DF
:10133C000599705409B0F0BD200D00202400002048
:08134C00010700002000002051
:1013540070B58021415821291AD102465632938A08
:10136400002B15D00168104C02E05B1E1D040FD049
:101374001588002D0DD0CD692D06F6D5056D2E8866
:1013840026408E62AD1C056515886D1E1580ECE740
:1013940070BD0120C0058A6882438A6008684022C3
:0C13A40002430A6070BDC046FF0100005B
:1013B00030B58023C15821290FD1024656321188F9
:1013C000002901680AD0036D1C88084D25408D62F4
:1013D000991C01651088401E108030BD0868984334
:1013E00008600868402202430A6030BDFF01000027
:1013F000F0B584B084214158222920D101465E31C4
:101400004E89320400D184E00246843203924B8834
:1014100003253540846D16D007687F6A1F4027700A
:101420000C88641E0C80846D641C84650F88002FFA
:101430000DD0012D23D1751E042E6AD380E00068E3
:101440001830082174E03546042E79D261E0012776
:101450003A020292026800921768029A9743009A31
:1014600017600196966802966C4F3740019E976010
:101470000027C7662027039A1760012DDBD0076875
:101480007F6A1F4027700C88641E0C80846D641C6A
:1014900084650F88002F05D0022D1BD1B51E042EA8
:1014A0004ED236E001273A02029202680092176893
:1014B000029A9743009A1760019595680295574FD5
:1014C0002F40019D97600027C7662027039A176069
:1014D000022DE3D005686D6A1D4025700C88641EDE
:1014E0000C80846D641C84650D88002D0ED101254F
:1014F0002A0207683D6895433D60BA68474D15402C
:10150000BD600025C5662025039A1560F51E042ED2
:1015100016D20A88002A0ED049898A420BD2414944
:10152000C1663E49491C006882680A4082602021E9
:1015300002680A43026004B0F0BD2D1F2E04E8D0FB
:101540000668766A1E4026700C88641E0C80846DC6
:10155000641C84650E88002E0DD106683768304AF9
:1015600017403760B7682D4A1740B7600026C66637
:101570002026039A16600668766A1E4026700C883C
:10158000641E0C80846D641C84650E88002E0DD151
:1015900006683768224A17403760B7681F4A174005
:1015A000B7600026C6662026039A16600668766A2B
:1015B0001E4026700C88641E0C80846D641C84653B
:1015C0000E88002E0DD106683768154A174037601F
:1015D000B768124A1740B7600026C6662026039AED
:1015E00016600668766A1E4026700C88641E0C80A1
:1015F000846D641C84650E88002E9ED10668376851
:10160000074A17403760B768044A1740B76000269A
:10161000C6662026039A16608FE7C046FEFFFFEFDE
:08162000FFFEFFFF85C000087A
:10162800F0B583B084214158222922D101465E3188
:101638004F893A0477D00246843202924B880326B7
:101648003E40856D046818D00197676A1F402F8057
:101658000F887F1E0F80AA1C009282650F88002FBA
:101668000FD0012E1DD1019F7E1E009D042F71D227
:1016780059E000681830082164E03E46042F69D21A
:1016880051E001273A02276897432760A268624F12
:101698001740A7600027C7662027029A1760012E07
:1016A800E1D0676A1F406F800F887F1E0F802A1D58
:1016B800009282650F88002F07D0022E019F15D156
:1016C800BE1E009D042F45D22DE001273A0227684F
:1016D80097432760A268504F1740A7600027C76646
:1016E8002027029A1760022E019FE9D0666A1E40E1
:1016F800AE800E88761E0E80AD1D85650E88002E84
:101708000ED1012636022768B7432760A668424FE4
:101718003740A760019F0026C6662026029A1660F9
:10172800FE1E042F16D20A88002A0ED049898A4242
:101738000BD23B49C1663849491C006882680A4097
:101748008260202102680A43026003B0F0BD361FA0
:101758003704E8D0676A1F402F800F887F1E0F80EC
:10176800AD1C85650F88002F0CD127682B4A1740C0
:101778002760A768284A1740A7600027C766202760
:10178800029A1760676A1F402F800F887F1E0F809C
:10179800AD1C85650F88002F0CD127681F4A17409C
:1017A8002760A7681C4A1740A7600027C76620273C
:1017B800029A1760676A1F402F800F887F1E0F806C
:1017C800AD1C85650F88002F0CD12768134A174078
:1017D8002760A768104A1740A7600027C766202718
:1017E800029A1760676A1F402F800F887F1E0F803C
:1017F800AD1C85650F88002FA9D12768074A1740B7
:101808002760A768044A1740A7600027C7662027F3
:10181800029A17609BE7C046FEFFFFEFFFFEFFFF3F
:0418280093C400085D
:10182C00F0B586B0012041044A4A13680B4313609B
:10183C0012680A40059205993D25474B02210491F7
:10184C005955464A1646183E1E609168444C214232
:10185C0006D19168434C214202D1316881433160F9
:10186C004821002402915C543E2101915C541F4696
:10187C003E377C70BC70FC703C717C7144210091D3
:10188C005C54194644314C708C70CC705C55364AA3
:10189C005C609C60DA601C611A462B46555D002D1D
:1018AC0001D13C2554551546049A0393EA542B4612
:1018BC000725ED013268AA439D6915433560274D14
:1018CC00294A6A612C615A69AA612A1F10602E4646
:1018DC00083E3268D20702D0326882433260029AE4
:1018EC009854019A98547870B870F870387178716F
:1018FC00009A985448708870C87003995854A96815
:10190C00AA688243AA602A6802432E46F025AA439D
:10191C0032600A229143B16031680C2291433160EC
:10192C00316811433160316D049A11430D2291439A
:10193C0031653C215C54FF2109020C4A13688B432E
:10194C00136040050A490860BFF34F8FBFF36F8FD8
:10195C0006B0F0BD40100240440E00201844014077
:10196C001111000044040000FFFF000014E400E02B
:04197C0080E100E026
:10198000F0B581B0017F012953D12B4C2168012989
:1019900005D10068406B2E490860022048E02168AC
:1019A000022946D101684A6B24490A600122530585
:1019B000234D2B60BFF34F8FBFF36F8F214B1E68FA
:1019C000F7680225AF43F760376A97433762376A93
:1019D0003762376A1C490F4206D1316A1B4F3942C0
:1019E00002D13168914331603E215A5444215A5406
:1019F000E94300680161164800681049096881429E
:101A000001D9081A03E0FED2081A124940181249F7
:101A10000860086800031149884208D2104807F09E
:101A200083FF0D48006801030E4809F0BBF803204E
:101A3000206001B0F0BDC046680F0020500F0020AC
:101A400080E100E0440E0020111100004404000079
:101A5000540F0020FFFF00006C0F0020405DC60007
:081A6000F0CC00084ECA00089A
:101A6800F0B58DB00120089005037B4F3D607B4C9D
:101A780020682168091A96290BD82168091A96291D
:101A880007D82168091A962903D82168091A9729BD
:101A9800EFD3734820210161226823689B1A962B93
:101AA8000BD823689B1A962B07D823689B1A962B6A
:101AB80003D823689B1A972BEFD30160206821680D
:101AC800091A96290BD82168091A962907D8216876
:101AD800091A962903D82168091A9729EFD33D6175
:101AE800FF2000065F490A688243089BD807101840
:101AF80008605D488021016005950BAD00200690C7
:101B0800A8705A482880DE033E61022228462946EA
:101B1800FFF7D8FA3E60262028703E610322284647
:101B28002946FFF7CFFA07963E60A8780A283DD1E4
:101B380020682168091A96290BD82168091A96295C
:101B480007D82168091A962903D82168091A9729FC
:101B5800EFD3079E3E610BAD22272F70032204921C
:101B680028462946FFF7AEFA3B480660422028700F
:101B780039480661A878072101402031697002229E
:101B880028462946FFF79EFA334806602F70074615
:101B98003E6128462946049AFFF794FA3E60A878E1
:101BA800800607D4324807F0BBFEFEE7314807F04D
:101BB800B7FEFEE735463E610BAF23203870064678
:101BC80004900322039238463946FFF77BFA2249EC
:101BD8000D604320019038700D61B878EF21014005
:101BE80079700222029238463946FFF76BFA1A4892
:101BF80005603E70056138463946039E3246FFF758
:101C080061FA1548056005610BAF049838703846CD
:101C180039463246FFF756FA0F4E3560019838704C
:101C28003561B8789F2101402031797038463946AE
:101C3800029AFFF747FA35600498387035613846DC
:101C48003946039AFFF73EFA3560B878800615D40E
:101C5800094807F065FEFEE7180000502400002040
:101C68001804005004E400E000E100E0460A000027
:101C780004C7000830CD00081FC700080BAD069840
:101C8800A8703420687051202870079F376102229D
:101C980028462946FFF716FA376031202870376141
:101CA800032228462946FFF70DFA3760A87834281A
:101CB80002D0F84807F034FE0BA8069A8270F6495D
:101CC800018009ADAA702A80376103222946FFF7EF
:101CD800F9F937602878FF2805D10BA8007809A9F9
:101CE800497881425DD00BA8069A8270EA49018042
:101CF80009ADAA702A80376103222946FFF7E2F965
:101D080037602878FF2805D10BA8007809A94978F9
:101D1800814246D00BA8069A8270DF49018009AD3E
:101D2800AA702A80376103222946FFF7CBF937606A
:101D38002878FF2805D10BA8007809A9497881429D
:101D48002FD00BA8069A8270D349018009ADAA70DA
:101D58002A80376103222946FFF7B4F937602878CB
:101D6800FF2805D10BA8007809A94978814218D025
:101D78000BA8069A8270C849018009ADAA702A800A
:101D8800376103222946FFF79DF937602878FF2835
:101D980000D09DE00BA8007809A94978814200D0BD
:101DA80096E009A885786020029005430BA8457045
:101DB800452103910170376109AE069931800222ED
:101DC80031460492FFF77EF9B44807603078FF285F
:101DD80005D10BA8007809A9497881425ED00BA8E3
:101DE800457003990170AD490F6109AE06993180BC
:101DF80002223146FFF766F9A84807603078FF28C5
:101E080005D10BA8007809A94978814246D00BA8CA
:101E1800457003990170A1490F6109AE0699318097
:101E280002223146FFF74EF99C4807603078FF28B8
:101E380005D10BA8007809A9497881422ED00BA8B2
:101E480045700399017095490F6109AE0699318073
:101E580002223146FFF736F9904807603078FF28AC
:101E680005D10BA8007809A94978814216D00BA89A
:101E7800457003990170894D2F6109AE069931802B
:101E880002223146FFF71EF92F603078FF283CD137
:101E98000BA8007809A94978814236D1804D049869
:101EA80068770BA8069B838028688168089A114385
:101EB800816079490B912A6A09A9012A45D0022A29
:101EC80040D0032A1A4643D1734A02600C9A3AE07A
:101ED8000899C802C906321F1268130402400B4051
:101EE8009A1842403260226823689B1AC82BF2D89D
:101EF80023689B1AC82BEED823689B1AC82BEAD8EC
:101F080023689B1AC82BEFD9E5E70899C802C906C8
:101F18002A1F1268130402400B409A1842402A6094
:101F2800226823689B1AFA2BF2D823689B1AFA2B8B
:101F3800EED823689B1AFA2BEAD823689B1AFA2B47
:101F4800EFD9E5E7574A026001E0574A0280026884
:101F5800081D03900BA882700899697709AFBB80A8
:101F680009934E4D079E2E6106223946FFF7AAF8BF
:101F78002E603878FF2820D10BA8007809A9497865
:101F880081421AD10BA8407809A98978814214D1D5
:101F98000BA8807809A9C97881420ED109A845798A
:101FA80001210398FEF798FAA84206D109A80079FA
:101FB80002990840602800D160E10498384D68779C
:101FC8000BA80021818028688268089B1A438260D8
:101FD800314A0B922A6A012A0BD0022A06D0032A18
:101FE8000A4609D12C4A02600C9A00E02D4A026088
:101FF80001E02D4A028002680BA882706B7709AF56
:10200800B9800991254D2E6106223946FFF75AF805
:102018002E603878FF2820D10BA8007809A94978C4
:1020280081421AD10BA8407809A98978814214D134
:102038000BA8807809A9C97881420ED109A84579E9
:1020480001210398FEF748FAA84206D109A80079A9
:1020580002990840602800D110E10498104D687773
:102068000BA80021818028688268089B1A43826037
:10207800094A0B922A6A012A18D0022A06D0032A92
:102088000A4616D1044A02600C9A00E0054A02602A
:102098000EE0C04638C9000825EC000018000050C2
:1020A800BC0E0020000025ECEC2500004F4A028001
:1020B80002680BA882706B7709AFB98009914C4D03
:1020C8002E6106223946FEF7FDFF2E603878FF287C
:1020D80020D10BA8007809A9497881421AD10BA808
:1020E800407809A98978814214D10BA8807809A978
:1020F800C97881420ED109A8457901210398FEF7D4
:10210800EBF9A84206D109A800790299084060288D
:1021180000D1B3E00498374D68770BA8002181807F
:1021280028688268089B1A438260334A0B922A6A9D
:10213800012A0BD0022A06D0032A0A4609D12E4AC0
:1021480002600C9A00E02D4A026001E0274A0280F2
:1021580002680BA882706B7709AFB9800991244D8A
:102168002E6106223946FEF7ADFF2E603878FF282B
:102178001FD10BA8007809A94978814219D10BA869
:10218800407809A98978814213D10BA8807809A9D8
:10219800C97881420DD109A8457901210398FEF734
:1021A8009BF9A84205D109A800790299084060283E
:1021B80064D004980F4D68770BA8002181802868A7
:1021C8008268089B1A4382600B4A0B922A6A012A8A
:1021D80016D0022A064F06D0032A0A4619D1064A03
:1021E80002600C9A00E0054A026011E0EC2500004C
:1021F80018000050BC0E002025EC0000000025EC63
:10220800014A0280014F03E0EC250000180000504D
:1022180002680BA882706B7709ADA98009913E61AD
:1022280006222946FEF74EFF3E602878FF2800D098
:1022380062E20BA8007809A94978814200D05BE2E4
:102248000BA8407809A98978814200D054E20BA8EC
:10225800807809A9C978814200D04DE209A845795A
:1022680001210398FEF738F9A84200D044E209A8F2
:10227800007902990840602800D03DE20E48CD3030
:1022880004900B900BAE02213046FEF725F9B07092
:102298000020069009900948079D056109AF0422AE
:1022A800304639460392FEF70DFF0448056038783A
:1022B800FF2818D104E0C04625EC000018000050A3
:1022C8000BA8007809A9497881420CD10BA840785D
:1022D80009A98978814206D10BA8807809A9C9780B
:1022E800814200D1A7E004980B900BAE0221304642
:1022F800FEF7F2F8B07006980990FE48056109AF3C
:10230800042230463946FEF7DDFEFA480560387883
:10231800FF2811D10BA8007809A9497881420BD16F
:102328000BA8407809A98978814205D10BA8807843
:1023380009A9C97881427ED004980B900BAE02217E
:102348003046FEF7C9F8B07006980990E94805616B
:1023580009AF042230463946FEF7B4FEE548056069
:102368003878FF2811D10BA8007809A9497881424B
:102378000BD10BA8407809A98978814205D10BA80F
:10238800807809A9C978814255D004980B900BAE82
:1023980002213046FEF7A0F8B07006980990D5489B
:1023A800056109AF042230463946FEF78BFEFE4828
:1023B80005603878FF2811D10BA8007809A9497859
:1023C80081420BD10BA8407809A98978814205D1AF
:1023D8000BA8807809A9C97881422CD004980B9061
:1023E8000BAE02213046FEF777F8B07006980990D8
:1023F800ED48056109AF042230463946FEF762FE12
:10240800E94805603878FF2800D095E10BA80078E6
:1024180009A94978814200D08EE10BA8407809A922
:102428008978814200D087E10BA8807809A9C9780A
:10243800814200D080E10BAE069DB580DB480B9051
:1024480002213046FEF748F8B07009AFBD80099503
:10245800D548079D0561062230463946FEF732FE0B
:10246800D1480560381D04903878FF2824D10BA87E
:10247800007809A9497881421ED10BA8407809A99A
:102488008978814218D10BA8807809A9C978814236
:1024980012D109AE7579012704983946FEF71CF860
:1024A800401B411E884103997156002900DA002714
:1024B8003843012800D061E10BAF069DBD80BB48C1
:1024C8000B9002213846FEF707F8B87009AEB580C0
:1024D8000995B548079D0561062238463146FEF73D
:1024E800F1FDB14805603078FF2824D10BA80078A9
:1024F80009A9497881421ED10BA8407809A9897891
:10250800814218D10BA8807809A9C978814212D1D3
:1025180009AE7579012704983946FDF7DDFF401BA0
:10252800411E884103997156002900DA0027384373
:10253800012800D022E10BAF069DBD809B480B907F
:1025480002213846FDF7C8FFB87009AEB580099575
:102558009548079D0561062238463146FEF7B2FDCB
:10256800914805603078FF2824D10BA8007809A984
:10257800497881421ED10BA8407809A989788142FF
:1025880018D10BA8807809A9C978814212D109AE5F
:102598007579012704983946FDF79EFF401B411EB7
:1025A800884103997156002900DA00273843012829
:1025B80000D0E3E00BAF069DBD807C480B90022164
:1025C8003846FDF789FFB87009AEB5800995764899
:1025D800079D0561062238463146FEF773FD7248AD
:1025E80005603078FF2824D10BA8007809A949781C
:1025F80081421ED10BA8407809A98978814218D157
:102608000BA8807809A9C978814212D109AE7579D9
:10261800012704983946FDF75FFF401B411E88419A
:1026280003997156002900DA00273843012800D0A1
:10263800A4E00BAF069DBD805C480B900221384694
:10264800FDF74AFFB87009AEB58009955648079D51
:102658000561062238463146FEF734FD52480560CA
:102668003078FF2823D10BA8007809A9497881423E
:102678001DD10BA8407809A98978814217D10BA8E8
:10268800807809A9C978814211D109AE777904986F
:10269800089D2946FDF720FFC01B411E884103996C
:1026A8007156002900DA069D2843012866D14B207F
:1026B8008000089AD102D2063B4F3B1F1B681D04BD
:1026C8000B401540EB184B403B6023682568EE1A19
:1026D80005466435AE42F0D82668F61AAE42ECD804
:1026E8002668F61AAE42E8D82668F61AAE42EDD940
:1026F800E3E7C046180000504B208000089AD1023A
:10270800D2063E46331F1B681D040B401540EB18CC
:102718004B40336023682568ED1A8542F2D8256856
:10272800ED1A8542EED82568ED1A8542EAD8256863
:10273800ED1A8542EFD9E5E74B208000089AD102CF
:10274800D206194F3B1F1B681D040B401540EB18A0
:102758004B403B6023682568EE1A05463235AE4289
:10276800F0D82668F61AAE42ECD82668F61AAE42B9
:10277800E8D82668F61AAE42EDD9E3E72068216862
:10278800091A96290BD82168091A962907D82168A9
:10279800091A962903D82168091A9729EFD30248FC
:1027A800059901600DB0F0BD1800005021EC000043
:1027B800F0B585B0B54807F0B3F8B54D01262E84BD
:1027C80037044B200002A861EF6128462A301E21F9
:1027D80009F014FBB820AF492950B420AE4929505C
:1027E800B020AE492950AC20AD4A2A50A820295023
:1027F800A4202A50A2207D2103912952C720C0433A
:102808004B30A02168529C20A64929509820A649FF
:10281800295096210220685294216E549021A34A8F
:102828006A508821A24A6A508021A24A6A502946E1
:102838001831A14A4A67A14ACA66A14A0021A14B98
:10284800AB64E96429656965AA65BC22A950D022F0
:10285800A950CC225A23AB522A46BC32516091600F
:10286800D160CA43984BC043984C29666966AA66EA
:10287800EA662C676A67AB67E867D8206860392022
:102888002870A868401CA860914C6068002806D58C
:10289800204608388F4901608F49016060688F4879
:1028A80000682168C9031FD421688D4A531C23601E
:1028B800114202D1216849036FD46068C00702D071
:1028C8006068B043606087480670874C2068874915
:1028D8000E700006400E401E8549086004A8FEF7E9
:1028E8005DF8002823D0FEE70399C9007B4A1268E7
:1028F800121A8A42E1D222683A42D5D0774A12683F
:10290800121A8A42D9D222683A42CDD0734A126842
:10291800121A8A42D1D222683A42C5D06F4A126846
:10292800121A8A42C9D222683A42DFD1BCE701971B
:10293800029620680006800B6E4E8419FF208702DD
:102948000CCD2046083DFDF79BFE0028FED16648C9
:102958000068800238403018D43008350834844282
:10296800EED35E4800685A490968019B1942029CE7
:102978003CD1574D29685A4A531C2B60114202D149
:102988002968490359D4E007514A51680143516005
:10299800506800F0B1F805B0F0BDB104039AD20058
:1029A8004E4B1B681B1A934287D223680B4284D074
:1029B8004A4B1B681B1A934200D37EE723680B42DD
:1029C80000D17AE7454B1B681B1A934200D374E782
:1029D80023680B4200D170E7404B1B681B1A9342D7
:1029E80000D36AE723680B42DAD166E70399C90086
:1029F8003A4A1268121A8A42C5D2354A12681A42ED
:102A0800B7D0364A1268121A8A42BCD2304A1268C3
:102A18001A42AED0314A1268121A8A42B3D22C4AEC
:102A280012681A42A5D02D4A1268121A8A42AAD2EE
:102A3800274A12681A42DBD19BE7A104039AD20005
:102A4800264B1B681B1A93429DD2214B1B680B42D5
:102A580099D0224B1B681B1A934294D21C4B1B68BB
:102A68000B4290D01D4B1B681B1A93428BD2184BFC
:102A78001B680B4287D0194B1B681B1A934282D2E2
:102A8800134B1B680B42DBD17DE7C0460ACB00081D
:102A9800E003002010270700320038FF54F248F402
:102AA8004C1D581B983AB036E02ED430B036D4308E
:102AB80080482800630069000A000200A08601001F
:102AC80040420F0090D00300007884C900D68AEAFB
:102AD8001020024023016745AB89EFCD2400002078
:102AE800FA830000900F0020E075FF1F8C0F002074
:082AF8005C0F002000F8FF074D
:102B0000F0B598B0DC4800680006800BDB4941183E
:102B1000481C1790881C1690C81C1590081D14900E
:102B2000481D1390881D1290C81D1190084608304A
:102B30001090084609300F9008460A300E9008465B
:102B40000B300D9008460C300C9008460D300B9061
:102B500008460E300A9008460F300990084610309B
:102B60000890084611300790084612300690084633
:102B70001330059008461430049008461530039031
:102B80000846163002900846173001900846183063
:102B900000900D4619350E461A36D720C743B8485F
:102BA000C019CB19D8229B5C8354179BDB199B5C03
:102BB000D9240355169BDB199B5CDA240355159B1E
:102BC000DB199B5CDB240355149BDB199B5CDC2429
:102BD0000355139BDB199B5CDD240355129BDB190A
:102BE0009B5CDE240355119BDB199B5CDF240355A2
:102BF000109BDB199B5CE02403550F9BDB199B5C4E
:102C0000E12403550E9BDB199B5CE22403550D9BCD
:102C1000DB199B5CE32403550C9BDB199B5CE424D0
:102C200003550B9BDB199B5CE52403550A9BDB19C1
:102C30009B5CE6240355099BDB199B5CE724035549
:102C4000089BDB199B5CE8240355079BDB199B5C05
:102C5000E9240355069BDB199B5CEA240355059B7D
:102C6000DB199B5CEB240355049BDB199B5CEC2478
:102C70000355039BDB199B5CED240355029BDB1979
:102C80009B5CEE240355019BDB199B5CEF240355F1
:102C9000009BDB199B5CF0240355EB199B5CF12432
:102CA0000355F3199A5CF223C2541B3700D076E720
:102CB00073498869734C2061888BA082C88BE0823D
:102CC000088C2083488CA083888CE083C88C208467
:102CD000088D6084488D7C22A052888D7E22A0526F
:102CE000C88D98221692A052088E9A221492A05251
:102CF000488E8C221292A052888EA0221592A05249
:102D0000C88EA8221792A0520A463832ECCAC86C64
:102D10001390086D1090486D0F90802022508422EF
:102D2000A3508822A55090231193E6509C26A751CA
:102D3000A425139B6351AC231393109FE7500F9B63
:102D4000A3678F6D9423E750085A5227E0538220DF
:102D5000085A5027E05308461830C06EE06588587E
:102D600020661298085A5422A0528E20085A5622E1
:102D7000A0521198085A5822A0529220085A5A225A
:102D8000A052C85C6422A0529620085A6822A05221
:102D90001698085AA0861498085AE086885B2087FF
:102DA0009E20085A60871598085AA087A220085AC2
:102DB000E087485B4022A052A620085A4222A05237
:102DC0001798085A4422A052AA20085A4622A05214
:102DD0001398085A4822A052AE20085A4A22A052FC
:102DE000B020085A4C22A052B220085A4E22A052BB
:102DF000B420085A6A22A052B620085A6C22A05267
:102E0000B820085A6E22A052BA20085A7022A05246
:102E1000BC200A582046C8304266C0228A588266C2
:102E2000C4228A58C266C8228A580267CC228A5AAB
:102E30007223E252D0228A5802660A6E15924B6EB5
:102E40000A46683264CA14964F6F8E6F1696CE6F1C
:102E500017964363159B036342648564C767149A9E
:102E600082672920C000169A225020184660C86840
:102E7000606018B0F0BDC046E075FF1F00F8FF07A6
:082E8000E003002028000020FF
:102E8800F0B59DB00390E24806F04AFDE1480068BD
:102E98000006800BE0494218501C1B90901C1A90A9
:102EA800D01C1990101D1890501D1790901D169049
:102EB800D01D159010460830149010460930139014
:102EC80010460A30129010460B30119010460C3004
:102ED800109010460D300F9010460E300E90104690
:102EE8000F300D90104610300C90104611300B909A
:102EF800104612300A9010461330099010461430CC
:102F08000890104615300790104616300690104667
:102F18001730059010461830049011461931FF23D8
:102F28009B02019300230293DC430094CF3CBB4BEC
:102F38001D191619D023F65CEE541B980619F65C79
:102F4800D127EE551A980619F65CD227EE5519982E
:102F58000619F65CD327EE5518980619F65CD4279F
:102F6800EE5517980619F65CD527EE5516980619EA
:102F7800F65CD627EE5515980619F65CD727EE5558
:102F880014980619F65CD8202E54139E3619F65C50
:102F9800D927EE55129E3619F65CDA27EE55119EA2
:102FA8003619F65CDB27EE55109E3619F65CDC27E1
:102FB800EE550F9E3619F65CDD27EE550E9E361936
:102FC800F65CDE27EE550D9E3619F65CDF27EE55CA
:102FD8000C9E3619F65CE027EE550B9E3619F65C0A
:102FE800E127EE550A9E3619F65CE227EE55099E52
:102FF8003619F65CE327EE55089E3619F65CE42789
:10300800EE55079E3619F65CE527EE55069E3619ED
:10301800F65CE627EE55059E3619F65CE727EE5571
:10302800049E3619F65CE827EE550E19F65CE9277A
:10303800EE557A4D1A3400D079E71990686D784EBC
:103048007065688D7085A88DB085686B1A90294663
:10305800383116C9686C1B90AF6CE86C1890286DF5
:103068001790688E7086A86DB065E88DF085288EFB
:1030780030861A987063B163F26334641B98706485
:10308800B7641898F06417983065039F012F04D02F
:10309800A869B061029805D105E04B200002B06133
:1030A800029800E0A88BB083012F03D1F78304D1E5
:1030B800632004E0E88BF083FAD07820285A2A8C21
:1030C80080217052012F06D0685888217050012F36
:1030D80005D10A2405E0534888217050F9E7842077
:1030E8002C5A8C201A903452012F06D07A242C5B4B
:1030F80082257453012F03D003E069248225745379
:103108003A463284012F029A444D0CD17284029AB5
:103118000DD1B284012F029A0ED1F284029A32851F
:1031280013E0EA6F12E06A8C7284029AF1D0AA8CDA
:10313800B284012F029AF0D0EA8CF284012F029A0D
:10314800EDD02A8D3285012FEBD1374A3446183419
:10315800E2660222012F1B9201D08622AA5A8E20F3
:1031680018903252314C012F00D06C5A9022B45230
:103178002F49012F0C4601D08A242C5B92201790EE
:1031880034523846012F01D1054601E01A9C2D5DC5
:103198009424355501281B98204D01D01898285A99
:1031A80096271A97F0530398012805D0AD5A98220C
:1031B800B552012804D106E0F84D9822B55202E034
:1031C800F4481799415A9A2571530398012802D057
:1031D800F0490C5B00E0F24C9C2174520128EE4847
:1031E80001D0EC48C05B9E27F053C720C443039826
:1031F800012802D0E748805A01E020464B30A0223F
:10320800B052039801281A9414D0E24A505B13E094
:1032180081C70008E075FF1F00F8FF07B804002009
:10322800E003002080482800A0860100B036000096
:10323800D43000007D20D74AA22417943053D94CAB
:1032480003980128204600D0505AA42116917052A4
:10325800D55BD549039A012A084600D02846A827F5
:103268001897F053D148012A024600D02A46A627CB
:10327800F253CF4A039D012D154603D0C54D17992A
:103288006D5AC949AA2417943553039D012DC54C7D
:1032980002D0C04C169D645BAC257453039C012C72
:1032A80001D0BC48C05BAE243053039F012F02D02D
:1032B800B8481899415AB0203152012F02D0B54967
:1032C800179A8A5AB227F2530399012903D0B149B0
:1032D8004A5B0D4601E03222AE4DB4217252039A88
:1032E800012A01D02A5B1A92B6221A9CB452039A78
:1032F800012A01D02A5A00E0AE4AB8203252039A75
:10330800012A01D0EA5B00E00722BA243253039D68
:10331800012D029A01D09F4A5258BC217250012DAA
:1033280002999A4C01D09B490958C0203150C420B9
:10333800012D02D09749095A00E05A21CC22B152F6
:10334800C821012D029A01D0924A5258F250029B8C
:10335800735033501B98C0439749984A3366736635
:10336800009FB766F76632677767B167F067894984
:103378008868401C886019997160B0603920307085
:10338800012D184601D08348007C3074012D02D0ED
:103398008048C06802900298F060894D68680028EB
:1033A80006D528460838874901608749016068685A
:1033B8008648006801211B910F042968C9031FD49E
:1033C8002968834A531C2B60114202D1296849039A
:1033D8006AD46868C0071B9A02D06868904368601E
:1033E8007C48027020687C490A700006400E401E26
:1033F8007A4908601CA8FDF7D1FA002823D0FEE717
:103408007D21C900714A1268121A8A42E1D22A68DB
:103418003A42D5D06D4A1268121A8A42D9D22A681D
:103428003A42CDD0694A1268121A8A42D1D22A6821
:103438003A42C5D0654A1268121A8A42C9D22A6825
:103448003A42DFD1BCE72068800201990840504920
:1034580044180CCE2046083EFDF712F90028FED18C
:103468004A48006880020199084049490818D43040
:10347800083608348442ECD3544800682968394235
:103488003BD12968524A531C2B60114202D129684A
:10349800490355D41B98C007696801436960686887
:1034A800FFF72AFB1DB0F0BD1B9989047D22D200CD
:1034B800464B1B681B1A93428BD22B680B4288D051
:1034C800424B1B681B1A934283D22B680B4200D1D4
:1034D8007FE73E4B1B681B1A934200D379E72B68A2
:1034E8000B4200D175E7394B1B681B1A934200D376
:1034F8006FE72B680B42DBD16BE77D21C900334AAC
:103508001268121A8A42C5D22A683A42B9D02F4A9A
:103518001268121A8A42BDD22A683A42B1D02B4A9E
:103528001268121A8A42B5D22A683A42A9D0274AA2
:103538001268121A8A42ADD22A683A42DFD1A0E74D
:103548001B9989047D22D200204B1B681B1A9342C9
:10355800A0D22B680B429DD01C4B1B681B1A9342B0
:1035680098D22B680B4295D0184B1B681B1A9342B4
:1035780090D22B680B428DD0144B1B681B1A9342B8
:1035880088D22B680B42DFD184E7C046E075FF1F65
:1035980000F8FF07B8040020B0360000E02E000055
:1035A800983A00004C1D000054F2FFFF581B000021
:1035B80048F4FFFF10270000007884C900D68AEA83
:1035C8001020024023016745AB89EFCD240000207D
:1035D800FA830000900F00208C0F00205C0F002061
:1035E800F0B591B00F90F14806F09AF9F04E3069B5
:1035F800F04DA861B08AA883F08AE883308B2884CC
:10360800B08B6884F08BA884308CE884708C288513
:103618007E20305AA8857C20305A688598200C90E6
:10362800305AE8859A200A90305A28868C200790CC
:10363800305A6886A0200B90305AA886A8200E9091
:10364800305AE8868024305904908422B058039078
:1036580088200590305802909020069030580190AC
:103668009C2008903358A42009903258AC200D9023
:103678003058B16F049FAF63039FEF63029F2F64BD
:10368800019F6F64AB64EA642865696594203158CA
:10369800A9655221715A29535021715A8222A9527F
:1036A800F16D2A461832D166316E059AA950542117
:1036B800715A079AA9525621715A8E22A952582135
:1036C800715A069AA9525A21715A9222A952642112
:1036D800715A29546820305A96216852B08E0C9934
:1036E8006852F08E0A996852308F08996852708F24
:1036F8009E216852B08F0B996852F08FA2216852B0
:103708004020305A099968524220305AA6216852FE
:103718004420305A0E9968524620305AAA216852DD
:103728004820305A0D9968524A20305AAE216852C2
:103738004C20305AB02168524E20305AB22168527B
:103748006A20305AB42168526C20305AB621685227
:103758006E20305AB82168527020305ABA21685207
:103768003046C830416EBC22A950816EC022A95093
:10377800C16EC422A950016FC822A9507221715A82
:10378800CC22A952016ED022A950016B0E91416B37
:103798000D91436C846C876FC06F0C902920C0001A
:1037A8003158301840680E9A2A660D9A6A66AB66D8
:1037B800EC662F670C9A6A67A967E867A868401CD7
:1037C800D8216960A860392028700F98002804D093
:1037D800794806F0A5F87068E860784C60680028B9
:1037E80006D5204608387649016076490160606848
:1037F800754E3068012739040F912168C9031FD419
:103808002168724A531C2360114202D1216849037E
:1038180069D46068C00702D06068B84360606C48CB
:1038280007706C4C20686C490F700006400E401EF3
:103838006A49086010A8FDF7B1F8002820D0FEE713
:103848007D21C9003268121A8A42E2D222680F9B8F
:103858001A42D5D03268121A8A42DAD222681A423B
:10386800CED03268121A8A42D3D222681A42C7D0FE
:103878003268121A8A42CCD222681A42E2D1BFE7D1
:103888000E9720680006800B554FC419FF2086024A
:103898000CCD2046083DFCF7F3FE0028FED14D482C
:1038A8000068800230403818D43008350834844223
:1038B800EED3454D2868414C21680F9A11420E9E5F
:1038C80034D12168414A531C2360114202D1216836
:1038D80049034BD4F0076168014361606068FFF7F2
:1038E8000BF911B0F0BDB9047D22D20033681B1A60
:1038F80093428ED223680B428BD033681B1A9342B3
:1039080087D223680B4284D033681B1A934200D3B2
:103918007FE723680B4200D17BE733681B1A934289
:1039280000D376E723680B42E0D172E77D21C90016
:103938002A68121A8A42CDD222680F9B1A42C0D036
:103948002A68121A8A42C5D222681A42B9D02A684D
:10395800121A8A42BED222681A42B2D02A68121AB1
:103968008A42B7D222681A42E2D1AAE7B1047D227C
:10397800D2002B681B1A9342ACD223680B42A9D001
:103988002B681B1A9342A5D223680B42A2D02B683E
:103998001B1A93429ED223680B429BD02B681B1A9A
:1039A800934297D223680B42E3D193E71FCB0008D9
:1039B80028000020E003002054CD00081020024019
:1039C80023016745AB89EFCD24000020FA8300006E
:1039D800900F0020E075FF1F8C0F00205C0F002067
:0439E80000F8FF07DD
:1039EC0010B5FFB083B0FD49086A086A0869096917
:1039FC004422C1B2AA296E9204D0D0433322CC29DE
:103A0C0004D004E05520C043332200E0D0430146EB
:103A1C005631049208D0C0B2CC2803D0BB2806D1B2
:103A2C00EF4802E0EF4800E0EF4805F077FF012691
:103A3C003102EA4C103C20686291084320607D20E2
:103A4C005D90C100E94800686C9106F0D9FF401EFA
:103A5C00010E37076F96B207119203223A92920722
:103A6C0063920029E24E22D1E2494860E24A106892
:103A7C00E24B1840639D28431060002088600720AB
:103A8C00086010681840119908431060DC486F9961
:103A9C000170B06B0843B063B06B084074907498BD
:103AAC00706B38437063706B38407490749868977F
:103ABC003A9B5902D34F3868509188430125A9028B
:103ACC004B91401838603868629908433860706DC3
:103ADC00182101437165CC48DB30396801403960ED
:103AEC00306838216A910840102201466792514093
:103AFC0072681A40022373935A4089184A424A4109
:103B0C00A9036591719569066991314608396B91E4
:103B1C00096800282ED0002A2CD10720C00281432E
:103B2C006B9A11601068629908431060B74801687D
:103B3C006B9A12684B9B1A4228D10268521A022ABD
:103B4C006FD86B9A12681A4220D10268521A022A54
:103B5C0067D86B9A12681A4218D10268521A022A54
:103B6C005FD86B9A12681A4210D10268521A022A54
:103B7C00DED956E0311F0A68A54B1A40659B1A43E3
:103B8C000A6000280BD09948006815E0984D281F52
:103B9C0001689F4A1140659A1143016032E0072089
:103BAC00C0026B9A11688143116010688004410F48
:103BBC009848C8408D49086091490E78002E119D97
:103BCC0000D135465D99C90006F01AFF401E8B499D
:103BDC00884226D887494860874A1068874B184026
:103BEC00639B184310600020886007200860002E3B
:103BFC0017D011460868814A104028430860804855
:103C0C0006707B4D28686A9A1040202801D000F07D
:103C1C0005FD686D28681040102801D000F0DCFD0F
:103C2C0068687198C003389020684007800F00D1F5
:103C3C004EE20720729000036D4B19680143196026
:103C4C007549F1391A680A401A606B990968699AC2
:103C5C00114200D0FEE1664B586B6899084007D1C1
:103C6C00596B689A11435963596B1140749174994B
:103C7C003968629A11433960719C21046091634EDA
:103C8C0031686E9D3A68629B1A4219D13268521A99
:103C9C00022A27D83A681A4212D13268521A022ADA
:103CAC0020D83A681A420BD13268521A022A19D813
:103CBC003A681A4204D13268521A022AE2D911E047
:103CCC006C99E8394A4A526D0A4021020A438A42E9
:103CDC00524901D000F0DFFC454B5A6D0A40629905
:103CEC000A435A650028424E04D101200007716B2B
:103CFC00814371633A98C043F16C0140F164119AAD
:103D0C00501EF16C01401143F164706860990843D6
:103D1C007060434805F002FEFDF782FD414F04241C
:103D2C003C60FDF77DFD52943C60719840057290AB
:103D3C00301F6D900068669000213B4E3B4C08E0B4
:103D4C000021709B98003A4A1150591C802900D1CF
:103D5C00C1E06D9A10680B462D490840709319020A
:103D6C004018106008E00A6802430A6072983149F2
:103D7C00086073990229E4D13868042862D10120C3
:103D8C0038603E21735C725D521E551EAA41012B98
:103D9C006F9B00D11346002B6E9DE7D1022272540B
:103DAC0072553168CB681343CB600A6A82430A624E
:103DBC000A6A02430A62204A914205D01F4A914284
:103DCC0002D01F4A9142CED1609AD31D8A681A4004
:103DDC00062ACBD003049A42C8D0C4E71020024074
:103DEC00DDC70008C2C70008F8C700082000002083
:103DFC000810024010E000E020ED00E0FFFFFF00A3
:103E0C00800F00200070004024FEFFFF24000020E3
:103E1C00FF80FFFF0024F400F0F1FFFFFFFCFFFF29
:103E2C006CC90008680F0020440E0020200F0020F1
:103E3C00EC07002000E100E00004004000400140DD
:103E4C00002C014038680328739993D138680328F3
:103E5C0000D075E77298B7490860BFF34F8FBFF376
:103E6C006F8F3568E86802218843E860286A719B87
:103E7C0098432862286A2862286AAF4A104207D100
:103E8C004B9844302A6A024202D128689843286031
:103E9C003E2033546E98335452983860A7480268C9
:103EAC00002A07D02068A64B1B681B03C018206093
:103EBC00092A03D8501CA14A10600AE000219F4A2D
:103ECC001160A04A11600A2106F09AFDA96A491CEA
:103EDC0041436E9D4EE77F2001026191669C0C4030
:103EEC006D9B1968984A114021431960401EFDD101
:103EFC00709078907790954CE06A02210F9108436E
:103F0C00E062E06A08407B907B98E06A5299084333
:103F1C00E062E06A08407B907B98E06A2021739114
:103F2C000843E062E06A08407B907B98E06A719EEF
:103F3C003043E062E06A30407B907B98F920470187
:103F4C00834807618349629888627696212037906E
:103F5C000004759070022790749074AD0846294641
:103F6C00FCF712FF70987790769075966697749719
:103F7C007748183864902946FCF706FF7696709FB0
:103F8C00759740205E907490734810382946FCF762
:103F9C00FBFE779776977596629874906D482946D4
:103FAC00FCF7F2FE7797769675967398749069483D
:103FBC0029463D46FCF7E8FE206B30432063206B1E
:103FCC00304074907498FF200E900002634A116880
:103FDC008143659801431160614827990160614CE8
:103FEC000720B1040702629A121D5F4B23605C929A
:103FFC006260A5605B97E76025616661A161679A65
:10400C00E26125626562A5620D90E06225636563DD
:10401C005D206D90205C320300280F9F0C92139151
:10402C0000D1A7E06D98275418681F465E9B9843F3
:10403C005F9738605A955995579556952F46134664
:10404C006798519058913146284653955C9D5495EC
:10405C005593EBE01D46296802227092114305230B
:10406C009943296041490D68384E36686A9A164062
:10407C00102E00D192E20E68761B3D4A964200D972
:10408C00E9E5324E36686A9A1640102E00D185E268
:10409C000E68761B364A964200D9DCE52B4E366804
:1040AC006A9A1640102E00D178E20E68761B304AC0
:1040BC00964200D9CFE5254E36686A9A1640102EE6
:1040CC0000D16BE20E68761B294A9642CCD9C2E528
:1040DC0020680221014305208143216023480168A7
:1040EC00236807221340022B00D1A2E503685B1A58
:1040FC001F4DAB4200D9AEE523681340022B00D113
:10410C0097E503685B1AAB4200D9A4E5236813401A
:10411C00022B00D18DE503685B1AAB4200D99AE5FE
:10412C0023681340022B00D183E50268521AAA427D
:10413C00D6D990E580E100E0111100000C0F0020B1
:10414C006C0F0020200F0020FF80FFFF08100240A2
:10415C0018000050000400501008005008E400E063
:10416C0000E100E0200D0020003001402400002080
:10417C00881300005C2000272754F449886B1043F7
:10418C008863886B104074907498C86A0125284322
:10419C00C862C86A28407B907897779776970220F8
:1041AC005F907590E02074907B9874A9649E304663
:1041BC00FCF7EAFD7F977E977D977C9538987B90EE
:1041CC007BA93046FCF7E0FD7398E14908606D98D7
:1041DC005F992154226810685E9988431060E80248
:1041EC00E36818430F210902884200D0A7625F924E
:1041FC005B9883425C9D00D80C9F5597D548F13055
:10420C0003405B93606B5A902046103007C858925D
:10421C00E2695192226A5692626A5992A26A579244
:10422C0062685492A2685392719E709F549A2A406D
:10423C00C94DAD1D539B1D40AA180F9B1840104330
:10424C0031400143589D2846279A104008436A99EB
:10425C00519B0B40034380200990569A02401A430D
:10426C006698E03066905799014011435F9B196046
:10427C005B9A55980243280C52990840104359995F
:10428C00679D2940014308225A9810400843586002
:10429C00F002D9698143D96127666D9826543C2078
:1042AC00AE4C129026542C206D9026542564739895
:1042BC006064A764E76427630D986063A06367621A
:1042CC00A762E661A6762783A54D201D0777A54832
:1042DC00183025606060A760E76007902061359218
:1042EC0062617D977C977B978097A06D002805D0A5
:1042FC00A868689F384200D1A7E0CEE000247894EB
:10430C00779401231805914A916B01439163916B4A
:10431C00014081918198D06A1843D062D06A1840CC
:10432C00709381908198D06A022171910843D06278
:10433C00D06A08408190819876940327759774937E
:10434C0074AD649E30462946FCF71EFD7694759735
:10435C007198749030462946FCF716FD7694759743
:10436C0004206790749030462946FCF70DFD769436
:10437C007597709874907C4806462946FCF704FDA6
:10438C00769475977198749030462946FCF7FCFC2E
:10439C00769475976798749030462946FCF7F4FC30
:1043AC007694759735987490649E30462946FCF740
:1043BC00EBFC769475971020749030462946FCF7E8
:1043CC00E3FC25216948719A4254694A0F32694BC2
:1043DC001D6815401D604D2252011D6815431D605E
:1043EC00654A05251560654F709E3E60C463465452
:1043FC000462F102802728C0046044608760629BDD
:10440C00C3600161739941618463C2638032026449
:10441C0046648464C46404652421083844544F49B8
:10442C0008658162564A50680E99884350600C9812
:10443C0054490860542049490C544848C465474CB9
:10444C002568A868689F384227D1A8684E49014062
:10445C003943A9604D4800684D4906F0D1FA400037
:10446C00801C80908098002817D08098401E8090E7
:10447C008098002811D08098401E80908098002849
:10448C000BD08098401E80908098002805D0809892
:10449C00401E809080980028E7D1A86838423D4E95
:1044AC0007D1A06D10210143A165E06D01210143ED
:1044BC00E165A868529908401022A16D11400818B6
:1044CC000F215B91C94364910028A16D679239D18A
:1044DC003148D9300140022071900143A165216916
:1044EC00AA68D20700D078E2236B002B0C9A00D17B
:1044FC0000220029729B02DA1A4B17330B40264616
:10450C00A4681C43337E9B032343747EE4031C4347
:10451C00B37E5F032743F4683C4314436D98325CCD
:10452C0052002243739FF45D012C00D011E2002B4A
:10453C0000D10CE20948836D3B438365C36D1C437A
:10454C00C46507E21143A165A8E2C0460810024009
:10455C00180000500F0E0000FA830000840D00209C
:10456C0000240140E8FFFF7F00040050E80D00200C
:10457C000080FFFF0800024000080240840802404F
:10458C0008E400E000E100E0E8FFFF6F20000020FD
:10459C00400D03002400002024FEFFFF2568729AC2
:1045AC001540032D00D2B8E02568709A15439D4341
:1045BC0025600A682368729D2B40022B00D1ACE069
:1045CC000B689B1AF44DAB4201D9FFF744FB2368EF
:1045DC00729D2B40022B00D19FE00B689B1AEE4D75
:1045EC00AB4201D9FFF737FB2368729D2B40022B9E
:1045FC0000D192E00B689B1AE74DAB4201D9FFF753
:10460C002AFB2368729D2B40022B00D185E00B689E
:10461C009B1AE14DAB42CDD9FFF71DFB686B689936
:10462C00084007D1696B689A11436963696B114043
:10463C00749174993968629A114200D099E0396882
:10464C0011433960F1490A683B68629D2B4200D0E6
:10465C008FE00B689B1A022B01D9FFF7E2FA3B683B
:10466C002B4200D085E00B689B1A022B01D9FFF777
:10467C00D8FA3B682B427CD10B689B1A022B01D9D0
:10468C00FFF7CFFA3B682B4273D10B689B1A022BB6
:10469C00DAD9FFF7C6FAED4F7A6D7B6D609C234338
:1046AC007B657B6DA3437B6513460B407B65D20713
:1046BC0001D1FFF711FB3268E44B5B6D9B0701D511
:1046CC00FFF70AFB33689B1ADE4CA34201D9FFF7B4
:1046DC0009FBDE4B5B6D9B0701D5FFF7FDFA3368D9
:1046EC009B1AA34201D9FFF7FDFAD84B5B6D9B07D0
:1046FC0001D5FFF7F1FA33689B1AA34201D9FFF7F2
:10470C00F1FAD24B5B6D9B0701D5FFF7E5FA3368E5
:10471C009B1AA342D0D9FFF7E5FACC4C2168814310
:10472C00216020688006400F00D1D5E020686A9A8D
:10473C0010400828C64800D1D4E021681140102947
:10474C0001D001F08BF8616803220A40032A00D0E3
:10475C00C04861684906490F491C06F051F9616867
:10476C004904490E48436168490F491C06F048F951
:10477C00B8E0B64A516D719B19435165B2490A684C
:10478C00B24D6B6D9B0758D40B689B1AAD4DAB4269
:10479C0001D9FFF746FAAD4D6B6D9B074DD40B68F5
:1047AC009B1AA84DAB4201D9FFF73BFAA74D6B6D95
:1047BC009B0742D40B689B1AA24DAB4201D9FFF761
:1047CC0030FAA24D6B6D9B0737D40B689B1A9D4D2D
:1047DC00AB42D5D9FFF725FA719800066B9A116890
:1047EC0081431160984801686B9A1268699B1A4260
:1047FC002FD00268521A022A01D9FFF712FA6B9ACB
:10480C0012681A4225D00268521A022A01D9FFF7FF
:10481C0008FA6B9A12681A421BD00268521A022AC2
:10482C0001D9FFF7FEF96B9A12681A4211D002688F
:10483C00521A022AD8D9FFF7F4F900286A9A01D043
:10484C00FFF7E8F971980007696B81436963FFF71B
:10485C00E1F97E4B5968804A0A40804951185960E9
:10486C007F49491C6B9D2A680A432A605968689ADB
:10487C001143596001686B9A1268699B1A4201D006
:10488C00FFF7CFF90268521A022A01D9FFF7C9F9CA
:10489C006B9A12681A4201D0FFF7C3F90268521AD8
:1048AC00022A01D9FFF7BDF96B9A12681A4201D09E
:1048BC00FFF7B7F90268521A022A01D9FFF7B1F9CA
:1048CC006B9A12681A4201D0FFF7ABF90268521AC0
:1048DC00022AD0D9FFF7A5F96B9800688004410F24
:1048EC005C48C840216889093C220A405D498958C6
:1048FC001F220A40D0405C4908605C4C2578002D92
:10490C00119E00D12E465D99C90006F079F8401E23
:10491C005349884201D9FFF79EF955494860554AD9
:10492C0010684F4B1840639B184310600020886040
:10493C0072980860002D01D1FFF78DF911460868B7
:10494C00474A1040304308602570FFF784F9609B9C
:10495C001A434948436A876AEE68484C3440002B36
:10496C00709103D0629EC03633403B4313432343C4
:10497C00EB60426863991140C36C129C045D012C7E
:10498C000CD1046C466C2643846C34430C431C439E
:10499C000121214303E0C0468813000019432A4E2D
:1049AC002B69374C1C400C432C610123DC07A242C1
:1049BC00314C709911D00324A407A2422E4C0CD078
:1049CC009B079A4209D05B9B9B041A402D4C26688E
:1049DC009E43B2181C4E2260274C6A690D9B9A4369
:1049EC00636B1A436A616A6920467024A243846B24
:1049FC00240114436C6101225405A14208D0002902
:104A0C0012D1A96A64980143A9620DE02400002028
:104A1C00A96A1948C16989001C311C240C4064998D
:104A2C00A140046E0C43AC6269690D9C2140994213
:104A3C002AD100211048C165816D1143719A9143AF
:104A4C0081652BE088130000240000200810024030
:104A5C0000127A000024F4008C80C11F020802208E
:104A6C00FFFFFF00C4BE000820000020800F0020C4
:104A7C0010E000E020ED00E0840D00200102DEFFDC
:104A8C0002FCFF1F08270140FC4CA16D10230B43B7
:104A9C0071988343A365E06D1043E06500277D9713
:104AAC0001247C947B947BAD2846FBF7C5FBA006C8
:104ABC001890801C7B902846FBF7BEFB6D94E0069B
:104ACC005C90001D7B902846FBF7B6FBEC487B9076
:104ADC002846FBF7B1FB689810307B902846FBF713
:104AEC00ABFBE8487B902846FBF7A6FBE6487B909F
:104AFC002846FBF7A1FBE5487B902846FBF79CFB7F
:104B0C00E3487B902846FBF797FBE24C7F20A7609D
:104B1C005790E0600E9820616761A761E76111987A
:104B2C00206271976762DC4802460C3A22602927A2
:104B3C00E15D002912D12821002363541121C902FF
:104B4C006160D64D696B4B9B19436963696B194066
:104B5C0074917499696D389B194369650F9906971F
:104B6C00E155CA215A9181615321816103685B0629
:104B7C006D9F27D4036880241C4304603368046849
:104B8C0064061FD43468E41A6C9DAC4214D80468D3
:104B9C00640617D43468E41AAC420DD80468640671
:104BAC0010D43468E41AAC4206D80468640609D4FC
:104BBC003468E41AAC42E2D90323B64C069D635523
:104BCC00036868E0C368B64C1C40C460C368C3602B
:104BDC000E9B4360579B1B0444681C434460036852
:104BEC00099CA3430360C3689B0626D40368A024D6
:104BFC00A343036033680468A40654D43468E41AED
:104C0C006C9DAC4214D80468A4064CD43468E41AE5
:104C1C00AC420DD80468A40645D43468E41AAC42FE
:104C2C0006D80468A4063ED43468E41AAC42E2D92F
:104C3C003A9B984C069D63552DE0C368739CA34327
:104C4C00C3600368A024A343036033680468A4060C
:104C5C0025D43468E41A6C9DAC4214D80468A406BC
:104C6C001DD43468E41AAC420DD80468A40616D4DA
:104C7C003468E41AAC4206D80468A4060FD434682D
:104C8C00E41AAC42E2D93A9B824C069D6355C36848
:104C9C00739C2343C3600E9B83617E4B11E0C368FE
:104CAC00739C2343C360C3687C07641E1C40C460B0
:104CBC00C368119C2343C3600E9B8361754B069C98
:104CCC001F5528240B941B5D012B00D15AE10F9B1F
:104CDC00704C069D63550B9BE7545A9B8361816115
:104CEC0003685B0627D40368099C2343036033687D
:104CFC00046864061FD43468E41A6C9DAC4214D862
:104D0C000468640617D43468E41AAC420DD80468FD
:104D1C00640610D43468E41AAC4206D804686406FD
:104D2C0009D43468E41AAC42E2D93A9A594B069D3C
:104D3C005A55026864E0C3687B041360BA04C36804
:104D4C009343C360C268C2600268099B9A430260C5
:104D5C00C268920626D40268A0239A430260326885
:104D6C0003689B0653D433689B1A6C9CA34214D8DB
:104D7C0003689B064BD433689B1AA3420DD8036877
:104D8C009B0644D433689B1AA34206D803689B063F
:104D9C003DD433689B1AA342E2D93A9A3D4B069D07
:104DAC005A552DE0C268739B9A43C2600268A023D7
:104DBC009A430260326803689B0624D433689B1ABA
:104DCC006C9CA34214D803689B061CD433689B1AB2
:104DDC00A3420DD803689B0615D433689B1AA342D3
:104DEC0006D803689B060ED433689B1AA342E2D9FB
:104DFC003A9A284B069D5A55C268739C2243C2604E
:104E0C000E9A826108E0C268739B1A43C2600E9AC4
:104E1C008261204B069D5F550F9A5A550B9A9F54F1
:104E2C005A9A82618161016849063BD40168099AEA
:104E3C001143016031680268520633D43268521A49
:104E4C006C9B9A4214D8026852062BD43268521AC0
:104E5C009A420DD80268520624D43268521A9A42E9
:104E6C0006D8026852061DD43268521A9A42E2D908
:104E7C003A99084A069BD154016873E0840D0020CE
:104E8C000800000C001000B00001002000020024FB
:104E9C0000040028900E00200C280040081002404E
:104EAC00BFFF8FFB01460839B34A0A600168099AB3
:104EBC0091430160C168890626D40168A022914300
:104ECC00016031680268920654D43268521A6C9BA5
:104EDC009A4214D8026892064CD43268521A9A42FA
:104EEC000DD80268920645D43268521A9A4206D8F6
:104EFC00026892063ED43268521A9A42E2D93A9922
:104F0C009E4A069BD1542DE0C168739A9143C160AF
:104F1C000168A0229143016031680268920625D491
:104F2C003268521A6C9B9A4214D8026892061DD4AD
:104F3C003268521A9A420DD80268920616D4326818
:104F4C00521A9A4206D8026892060FD43268521A44
:104F5C009A42E2D93A99894A069BD154C168739B0B
:104F6C001943C1600E998161104608E0C168739ABB
:104F7C001143C1600E9981618048069947540B9981
:104F8C00719A4254F64D286B0C9B18432863F54CD0
:104F9C0027620D9AA260679DE5600E982061719F53
:104FAC006761A7610230A080F4480146083921608E
:104FBC00EB49096B194074917499617F002900D1F8
:104FCC0021770F9B6377C26001682943359A91431F
:104FDC000160216981600168602291430160016870
:104FEC00099A914301606D9D65776802E44A1080CF
:104FFC001446C834E765A76545204A908100F843FC
:10500C000591505264990F316164A1644721169146
:10501C008900159150528F2149001491505223212F
:10502C00C900089150528D214900029150521381B0
:10503C00558105203690908107982062D148173011
:10504C0059906062D0482081411E55916181606108
:10505C006198FF30A061C12040002D901752106E56
:10506C00CA4B58430699C90050506491511863912A
:10507C00C0174860D06D5843A067C0177094E067A4
:10508C00C348806B0006800BC249405C382815D0A1
:10509C00392809D0FF281DD1BF4804F03FFCB8497E
:1050AC004F800E98C88118E0BC4804F037FCB44916
:1050BC004D803920C881FDF71DFD10E0B84804F083
:1050CC002DFC0220AE4948806A98C8810020FDF76B
:1050DC00D5FE04E03A995180D081FDF767FBB148C9
:1050EC0004F01CFCFDF706FDAF48006840061AD41E
:1050FC0030683168091A32290BD83168091A3229FB
:10510C0007D83168091A322903D83168091A3329AA
:10511C00EFD3A5480068400605D4A44804F0FEFB74
:10512C000120FDF7ABFEA248A24A02600C24A24B60
:10513C0054619761D7611762576297629049086909
:10514C0013605060888A9D4A531EC98ACA1E92B247
:10515C0010939A422A4600D30A46022801D3092109
:10516C0000E00A2192B200284B9D0C9B0AD001282A
:10517C0006D1509D06E0C04616241800900E002063
:10518C003D463B4688188B4961938B605F950D615A
:10519C00012A00D0669F874D6697EF6005F0A6FB4D
:1051AC00874B719F3A4606F0B5FF05F017FB5890F8
:1051BC00099AA85800283E4638463B4639467E4F49
:1051CC0041D17C2000247B490C546549886B659A3D
:1051DC0010438863886B104074907498C86A0225D9
:1051EC002843C862C86A28407B9078947794012041
:1051FC00769075955E9874907B9874AE714F384626
:10520C003146FBF7C1FD78947794769475958020A0
:10521C00749038463146FBF7B7FD099A6A4B18690A
:10522C006A49084018616A485C990160614DA86838
:10523C006190E868669028695F906C69AB69E96970
:10524C00286A6E6A2F685C930B4624215691594D3F
:10525C00A9503A68012154918A433A605F990C43F2
:10526C0061990C436A6E22433C685A4D25401543A4
:10527C0065931D433D603A9A12037C68944366998A
:10528C000C437C605C990843BA68534B134003434E
:10529C00BB60F86A5B9A90433043F8624F48874290
:1052AC003B46354609DC4E4883424E4E679917D033
:1052BC004D4883423F4F1BD010E04C488342494E2F
:1052CC003C4F679914D03C48834207D12448C06CAA
:1052DC008007000F464A1058719009E0719107E061
:1052EC001F48C06C0C220240414880587190314FCD
:1052FC0067936D98C003389A6599914226D171993C
:10530C00082900D95AE149007944898849008F4419
:10531C0008005501D80055018A0055015501550169
:10532C00E400344800680E490968890A1C220A40C6
:10533C00314989581F220A40D0400B2D00D2F9E088
:10534C000B2D629900D1F8E00121F6E07199082942
:10535C0000D933E104A24900515A49008F44C04698
:10536C0008100240BC0E00204E002E01B7002E018A
:10537C008A002E012E012E01C300C04608300240C7
:10538C0028000020E8FFFF7F0080FFFFF0F1FFFF07
:10539C00A875FF1F00F8FF0756C90008DDCA0008F2
:1053AC003AC70008A0C7000810080050AFC7000893
:1053BC00B8050020940A002000380140FFFF0000CF
:1053CC0000000C400004005008E400E0FFFFFF0068
:1053DC0000E100E0F369FFCFFFF4FF11FF4B004049
:1053EC00004400402400002000480040004C0040D5
:1053FC0088BE00082000002004BF0008FA4800689E
:10540C00FA490968890A1C220A40F94989581F225D
:10541C000A40D0400B2D00D2A9E00B2D629900D18F
:10542C00A8E00121A6E0F14A10688006400F78D070
:10543C0010686A9B18400828EE4878D0116819400B
:10544C00102900D019E2516803220A40032A00D027
:10545C00E948E64C61684906490F491C05F0D0FA49
:10546C0061684904490E48436168490F491C05F0BD
:10547C00C7FA5CE0DD4A10688006400F6ED01068F9
:10548C006A9B18400828DB486ED011681940102917
:10549C0000D0FFE151683A9A1140032900D0D64858
:1054AC00D24C61684906490F491C05F0A9FA61689C
:1054BC004904490E48436168490F491C05F0A0FA9C
:1054CC0052E00B2D15D2A800CC49095814E00B2D35
:1054DC0014D2A800C949095813E00B2D13D2690046
:1054EC00C74A515A13E00B2D17D26900C44A515ABE
:1054FC0040E0629900D00121BF481EE0629900D0C3
:10550C000121BD4836E001210B2D00D1090205F027
:10551C0077FA41007C68600814E000D19BE1549953
:10552C0028E06B9800688004410FB348C8400B2DED
:10553C0000D305E7A900B14A515805F061FA4000C3
:10554C007C6861080818214605F05AFA60991039F0
:10555C00014033D00007400F084316E06B980068F9
:10556C008004410FA448C8400B2D00D355E7A90077
:10557C00A24A515805F044FA7C6861080818214683
:10558C0005F03EFA80B20F2818D9679AD060002532
:10559C009C48B866FD663D67B86A002870D0C107A4
:1055AC0013D181071BD4410723D401072BD4C10687
:1055BC0032D481063AD4410642D457E09148B866B9
:1055CC000020F8663867739FD9E00121490413461F
:1055DC0052688A43F96A114359608107E3D5012166
:1055EC000904679B5A688A43396B11435960410718
:1055FC00DBD501218904679B5A688A43796B114377
:10560C0059600107D3D5679B5968559A1140BA6BFD
:10561C000A435A60C106CCD501210903679B9A68DD
:10562C008A43F96B114399608106C4D50121490362
:10563C00679B9A688A43396C11439960410615D56A
:10564C000121090571953546679E72688A437B6C0A
:10565C001A4372602E46719D8B4207D13A994905C7
:10566C00679B5A688A43B96C114359600006679A64
:10567C0006D50120C00451688143F86C0843506082
:10568C000127F805516801435160106818990843C7
:10569C0010603A984002D63060435B4905F0B0F98F
:1056AC005A498C42589A00D3421C5948401C679C5A
:1056BC006169014011436161206838432060882092
:1056CC0054490D5030682168090722D5E169729A56
:1056DC0011421ED131680A1A6999491E8A423ED874
:1056EC00E269729B1A4214D13268121A8A4236D875
:1056FC00E2691A420DD13268121A8A422FD8E26935
:10570C001A4206D13268121A8A4228D8E169194223
:10571C00E0D0216849072AD5E169490227D4B905A7
:10572C003268131A699A521E934218D8E3690B42D5
:10573C001DD133681B1A934211D8E3690B4216D161
:10574C0033681B1A93420AD8E3690B420FD13368B2
:10575C001B1A934203D8E2690A42E1D007E02E48B3
:10576C003B30216801402160A068B843A0600998D3
:10577C002849739F0F507C200D5484200F502748CC
:10578C0000687C210A91445C01467C31012C0ED0CE
:10579C00569A4A600268136815680126B54315606D
:1057AC007507AB431360002242660A704F608A682B
:1057BC00202A0C9E14D103465C338268B2420DD170
:1057CC00012C0DD00469002C0AD00E9C9C80012465
:1057DC0024025C801C80124C84656AE0012C23D16D
:1057EC00104805F0D9F9FEE720000020081002400F
:1057FC0004BF000800127A000024F40098BE0008D0
:10580C0030C400080100010040420F00014B0000B1
:10581C00FFFFFFFE940A002024FEFFFFB8050020C6
:10582C00DF050020E0C80008012425025D801D80F2
:10583C00E54D8565002A07D02407A24209D10469E9
:10584C00002C04D03F2433E00469002C2FD0579C4B
:10585C002EE000242CE0549909028BE620681040BD
:10586C002028389801D1FFF73DF8206810401828FF
:10587C0000D1A4E10020FFF735F81068184020286B
:10588C00389800D153E610681840182800D1D0E1A0
:10589C0000204CE6106818402028389800D163E6A8
:1058AC0010681840182800D1C6E100205CE60E9C58
:1058BC009C8000247394CC60222439948C600468FE
:1058CC00A56801273D43A56058977F07456E019752
:1058DC00BD4204D101252D029B89AB420ED9B242A7
:1058EC0003D10269002A00D1CEE0D54AD54E00235F
:1058FC000B70C266629F2037224611E0B24203D180
:10590C000269002A00D125E1CF4BCE4E689F22467A
:10591C00083200250D70C366206862990843206028
:10592C0026206590739D3554106838431060F561DE
:10593C00B584358430461C308571C44F388804F0EA
:10594C00C5FF7321CC05214604F088FDC04F3946B4
:10595C0004F084FD04F030FF0646BE480660BB48E8
:10596C00408C04F0B3FF214604F078FD394604F076
:10597C0075FD04F021FF801BB7490860542774950E
:10598C00B64BD85D5899CA05039201281C68349708
:10599C0002D1A068B24EE6E2D955A068A168C90749
:1059AC00AF4E23D00F99084020D1A06836990840FB
:1059BC00012812D1A068AB4908400F990843A06098
:1059CC003A9820603068A168C9070FD03168091A6D
:1059DC000329F8D3A168C907F5D0A04A906D10210E
:1059EC0001439165D06D58990843D065A068C007F4
:1059FC009A4A906D40D19C49D93108400F9908437F
:105A0C009065E1689948001FE2680240E260A06876
:105A1C00944A104010181830A0603898C01C0840E8
:105A2C0072902146B431924AA368002B2ED5749BF8
:105A3C005B1C7493749B934200D9B7E1A368002B51
:105A4C0024D5749B5B1C7493749B934200D9ADE179
:105A5C00A368002B1AD5749B5B1C7493749B9342A4
:105A6C0000D9A3E1A368002B10D5749B5B1C749325
:105A7C00749B9342D8D999E1102108437749739AC2
:105A8C00CA55886510469AE17A4A2FE70B68A568D3
:105A9C007448054045191835A56057980340A5680A
:105AAC00002D24D5749D6D1C7495749D954200D960
:105ABC007CE1A568002D1AD5749D6D1C7495749DA0
:105ACC00954200D972E1A568002D10D5749D6D1C0E
:105ADC007495749D954200D968E1A568002D06D592
:105AEC00749D6D1C7495749D9542D8D95EE10D68BA
:105AFC00A6685C48064086191836A660584E57981A
:105B0C000540EB18A568002D26D5749D6D1C749569
:105B1C00749D954200D949E1A568002D1CD5749D52
:105B2C006D1C7495749D954200D93FE1A568002DBC
:105B3C0012D5749D6D1C7495749D954200D935E1F8
:105B4C00A568002D08D5749D6D1C7495749D9542A7
:105B5C00D8D92BE1484BD8E60D68A66841480640D9
:105B6C0086191836A6603E4E579805405B19A568F5
:105B7C00002D2BD5749D6D1C7495749D954200D988
:105B8C0014E1A568002D21D5749D6D1C7495749D30
:105B9C00954200D90AE1A568002D17D5749D6D1C9E
:105BAC007495749D954200D900E1A568002D0DD522
:105BBC00749D6D1C7495749D9542D8D9F6E05D98D2
:105BCC000002FEF78FFEC046DF0500200D68A668B8
:105BDC002448064086191836A660214E5798054071
:105BEC005B19A568002D49D5749D6D1C7495749D29
:105BFC00954200D9DAE0A568002D3FD5749D6D1C47
:105C0C007495749D954200D9D0E0A568002D35D5CA
:105C1C00749D6D1C7495749D954200D9C6E0A56861
:105C2C00002D2BD5749D6D1C7495749D9542D8D9FF
:105C3C00BCE05D9800027AE45D98000294E4C046F2
:105C4C0085C00008B8050020F1130008A875FF1FD7
:105C5C0000803B45280F0020240F0020840D0020DD
:105C6C0024000020E8FFFF7F24FEFFFF0080FFFFE1
:105C7C00FFF1020093C40008291600080D68A668FD
:105C8C00E848064086191836A660E74E5798054036
:105C9C005B19A568002D22D5749D6D1C7495749D9F
:105CAC00954200D982E0A568002D18D5749D6D1C15
:105CBC007495749D954279D8A568002D0FD5749D67
:105CCC006D1C7495749D954270D8A568002D06D5F1
:105CDC00749D6D1C7495749D9542DAD966E00D68BF
:105CEC00A668D048064086191836A660CE4E57983E
:105CFC0005405B19A568002D21D5749D6D1C74950C
:105D0C00749D954252D8A568002D18D5749D6D1CB4
:105D1C007495749D954249D8A568002D0FD5749D36
:105D2C006D1C7495749D954240D8A568002D06D5C0
:105D3C00749D6D1C7495749D9542DBD936E00D688D
:105D4C00A668B848064086191836A660B64E57980D
:105D5C0005405819A568002D01D403F023F8749D53
:105D6C006D1C7495749D954220D8A568002D01D4A6
:105D7C0003F018F8749D6D1C7495749D954215D89C
:105D8C00A568002D01D403F00DF8749D6D1C74955D
:105D9C00749D95420AD8A568002D01D403F002F831
:105DAC00749D6D1C7495749D9542D3D900209F4BA6
:105DBC00D855996D10220A430F998A439A65411E52
:105DCC0048424841A16849076F9900D4014600290F
:105DDC0000D0C8E058999548C155E068C0070CD16F
:105DEC00A068C00706D0A0688E4908400F990843E8
:105DFC005899A060E0680843E06073987490A068BC
:105E0C00C00741D187482F30A168014209D0874A89
:105E1C00906D102101439165D06D58990843D06560
:105E2C00A1E0A0687F49084058990843A0608048C9
:105E3C0000680399084221D07E4800687E4904F02E
:105E4C00DFFD401C74907498002817D07498401E85
:105E5C0074907498002811D07498401E74907498A3
:105E6C0000280BD07498401E74907498002805D0AC
:105E7C007498401E749074980028E7D16B48407E4B
:105E8C00012801D002F074FF684A739BD3556B480C
:105E9C00FF30916D0140629801439165D3651C23DD
:105EAC002360106D6649674A674DC56202634163A2
:105EBC00616810220A4362605699415C01294CD0FA
:105ECC0001462431589D0D704A78012A41D10F9A10
:105EDC004A707399C16301680A68AA430A60826CAC
:105EEC00C56C5560026D002A02D0456D866D6E60E2
:105EFC0025464035066C1E40589BB340534E361F0A
:105F0C0037681F43376009234B608668504B102E4F
:105F1C001F4600D02F468F60102E00D01D46CD603E
:105F2C000B680E251D430D60406C0368609D2B4271
:105F3C003D4E03D00368629D2B430360002A03D0BF
:105F4C001068629B184310600868589A10430860E8
:105F5C0003E0739A0A700999C163A068314908403B
:105F6C0052990843A06030683168091A64290BD82B
:105F7C003168091A642907D83168091A642903D8C9
:105F8C003168091A6529EFD3FBF768FD314803F036
:105F9C00C5FC70983049C1878187304F388B0028F9
:105FAC0031D05898C002002104E0491C2B4A128BB6
:105FBC00914228D22A4A106033683268D41A629A05
:105FCC005E3294420BD83468E41A944207D8346891
:105FDC00E41A944203D83468E41A9442EDD9204B65
:105FEC00186133683468E41A9442DED83468E41AD1
:105FFC009442DAD83468E41A9442D6D83468E41A55
:10600C009442EFD9D1E7E12000016B904D2017901D
:10601C0040010021134D5F3019906D9169915F9192
:10602C002BE0C046E8FFFF7F24000020840D0020F9
:10603C000827014020000020400D0300FFEFFFFF68
:10604C0047C4000831C00008D10100080800024014
:10605C00E00E002034CB0008FFFF000028000020D9
:10606C001800005001A0000000207399705030758A
:10607C0084209249399A0A5039466A9190480068AE
:10608C00012801D000F0F8FB00258D4805608D4FEC
:10609C0038688109401A8C4FB9684418A1098B489B
:1060AC004843000CC8228A4B98528A4804F0A8FC3A
:1060BC00709E70803868C1177288002304F060FCF1
:1060CC000622002304F05CFC0904000C4018F0606C
:1060DC007C480460804800687C6880491731739163
:1060EC0088426F9908D0411C7B4A116019998842EB
:1060FC0001DC002100E001217291794A1068010A4B
:10610C00401A00191060000A718800230A0C050C53
:10611C002F46574380B242438EB270436E43150CE8
:10612C00110440187D41310C3204709E10186941E5
:10613C00062204F025FC0904000C4018306172980A
:10614C0000280BD030697169884201DD30697061BB
:10615C003069B169884201DA3069B0615A985C4E95
:10616C00305A0025210C020C13464B4380B241439C
:10617C00A4B2604354430A0C090440185A41210C40
:10618C0023041818514106222B4604F0F9FB09048C
:10619C00000C40186521890070504B49C868514A61
:1061AC0012680969739B9A4202D0521C4D4B1A60BB
:1061BC00401A04F04FFB04460E46709F788804F09A
:1061CC0095FB2246334605F0A5FF2A46464B05F0C3
:1061DC00A1FF2A46454B04F09DF9454A454B04F076
:1061EC0099F904460E4694203949085804F032FBBC
:1061FC002A46414B04F08EF92246334605F08AFFBD
:10620C0004F086FA19210A017292314988503A69D0
:10621C00D317F869C11704F0B3FB5D9AD2002B4673
:10622C0004F012FC386435480068396E081ACD2128
:10623C004900274A50523249081D7C2205F0E6FDE0
:10624C00304E301D31467C2205F0E0FD729820491D
:10625C00085872902A490860F868539030602A46B2
:10626C002B46739806E02D1D802D73913A463346CC
:10627C00204619D023494959CC176140091B91423A
:10628C000F4600DC1746739A914200DB11461C4AFC
:10629C005259D4176240141B9C42264600DC1E4601
:1062AC008442E0DB0446DEE7781AC1174840401A06
:1062BC005190642828D3002527E0C046940A00207A
:1062CC00080F00204C0F0020E00E0020E40C000012
:1062DC00280000200000B80B700F0020E8FFFF7FA3
:1062EC00740F0020580F00200000F03E00004440C6
:1062FC00FCA9F1D24D62403F80842E41600F0020FA
:10630C00200C0020200B00200125094F301BC11749
:10631C004840441AF86D6821795A04F071FBC11792
:10632C00890F40188010509484426F9803DB01E071
:10633C002800002028460028014D03D09CE2C046CE
:10634C0001A00000074842688368981AC1174840AA
:10635C00401A72992492511ACA175140891A8842CC
:10636C0003DC01E0200C002008460449CC68E11A4B
:10637C00CA175140891A814203DC01E0200C00202D
:10638C00014604480569281BC2175040801A8842F0
:10639C0003DC01E0200C0020084604494E69711B07
:1063AC00CA175140891A814203DC01E0200C0020FD
:1063BC00014604488769B81BC2175040801A8842AE
:1063CC0003DC01E0200C002008460549C9694F9107
:1063DC00C91BCA175140891A814204DC02E0C0462D
:1063EC00200C002001460548026A4F984E92101A64
:1063FC00C2175040801A884203DC01E0200C0020B8
:10640C00084605494A6A4E994D92511ACA1751408D
:10641C00891A814203DC01E0200C0020014605486A
:10642C00826A4D984C92101AC2175040801A8842BA
:10643C0003DC01E0200C002008460549CA6A4C998F
:10644C004992511ACA175140891A814203DC01E062
:10645C00200C002001460548026B49984892101AFE
:10646C00C2175040801A884203DC01E0200C002047
:10647C00084605494A6B48994792511ACA17514028
:10648C00891A814203DC01E0200C002001460548FA
:10649C00826B47984692101AC2175040801A884255
:1064AC0003DC01E0200C002008460549CA6B469924
:1064BC004592511ACA175140891A814203DC01E0F6
:1064CC00200C00200146FE48026C45984492101A9C
:1064DC00C2175040801A884200DC08465490F84895
:1064EC00426C4498101AC1174840411A5498814282
:1064FC00269100DC01465591F148806C4390801A3E
:10650C00C1174840411A55988142289100DC014638
:10651C005691EB48C16C43984291081AC1174840F8
:10652C00411A56988142299100DC01465791E44862
:10653C00016D42984191081AC1174840411A579869
:10654C0081422A9100DC01465C91DD48416D419805
:10655C004091081AC1174840411A5C9881422B910E
:10656C0000DC01466191D648816D40983F91081A34
:10657C00C1174840411A619881422C9100DC0146B8
:10658C006691CF48C16D3F983E91081AC11748409B
:10659C00411A669881422E9100DC01462097679142
:1065AC00C748016E3E983D91081AC1174840411AE0
:1065BC00679881422F9100DC01462F466891C048B4
:1065CC00416E3D983C91081AC1174840411A689891
:1065DC008142309100DC014625467191B848816EAC
:1065EC003C983B91081AC1174840411A7198814256
:1065FC00319100DC014673911F922196B048C26E16
:10660C003B98101AC1174840441A7398844232942C
:10661C0000DC04462593AA48036F1E92991ACA17E8
:10662C0051408E1AA642314600DC21463394239504
:10663C00446F1D93E21AD3175A40D31A8B421A4651
:10664C0000DC0A462297856F1C942C1BE7177C40B4
:10665C00E41B9442274600DC1746C06F1B951A902A
:10666C00401BC5176840401BB842964D00D903E14A
:10667C00944200D900E18B4200D9FDE03398864268
:10668C0000D9F9E073983299814200D9F4E07198FD
:10669C003199814200D9EFE068983099814200D954
:1066AC00EAE067982F99814200D9E5E066982E9927
:1066BC00814200D9E0E061982C99814200D9DBE05D
:1066CC005C982B99814200D9D6E057982A9981423F
:1066DC0000D9D1E056982999814200D9CCE055983F
:1066EC002899814200D9C7E054982699814200D854
:1066FC00C2E0519804F0AEF804460D46509804F0F0
:10670C00A9F802460B462046294603F003FF002257
:10671C006D4B05F0FFFC03F0FBFF14996B4B5852CB
:10672C002520C000185871905720C000739019187C
:10673C007298C8676722D00072901B185398D8675C
:10674C0024988867624A151DE0CD106954696194DC
:10675C0094696694D4696794146A68949D67259DBE
:10676C004D675E67239D0D671F67229DCD66D866BA
:10677C0021988866619898665648719C04602098A8
:10678C004866669858664F980866679818664E98DB
:10679C00C8656898D8654D988865506A946AD56ABA
:1067AC00166B576B6697976B6797D76B6897176CD9
:1067BC00719798654C9848655C65499808651D65A6
:1067CC004898C864DE6447988864669898644698CC
:1067DC0048646798586445980864689818644498A5
:1067EC00C863DF631F988863506C946CD56C166D0E
:1067FC00576D6697976D6797D76D6897176E7197FA
:10680C009863439848635C63429808631D6341989E
:10681C00C862DE6240988862669898623F984862C7
:10682C00679858623E980862689818623D98C861EB
:10683C00DF613C988861506E946ED56E166F576F01
:10684C006897976F7197D26F98613B9848615C61BC
:10685C001E9808611D611D98C860DE60194D1C985A
:10686C008860689898601B9848605F60174F1A980A
:10687C007399785072983A5017480068012801D0E3
:10688C0000F0CEFC74A8002101720226134B5E7737
:10689C00186882680124224382607591104A7492B0
:1068AC001A6A012A20D0022A06D0032A0A461ED1CF
:1068BC000B4A0260002200E00A4A026016E0C04661
:1068CC00200C002001A0000000408F402800002078
:1068DC00200B0020600F0020040F0020BC0E0020B5
:1068EC0012EC0000000012ECC64A0280026874A888
:1068FC008270C54A739454777BAC21727C917B91E6
:10690C00389FC24D2F6109222146FAF7D9FB2F601F
:10691C002078FF28BE4D5AD174A800787BA94978FD
:10692C00814254D174A840787BA9897881424ED198
:10693C0074A880787BA9C978814248D12F46B24D82
:10694C006E777BA8007A2A68936801210B439360C9
:10695C002B6A012B17D0022B0AD0032B1CD17C9B4A
:10696C0013607D9B13607BABDC6814601B690CE0CF
:10697C007BABDC887C9E3604341914605B897D9C6F
:10698C002404E31801E07C9B1BBA1360126869773E
:10699C0082423D4605D01AE00022697782423D468C
:1069AC0015D17BA80079CC21014084290FD17BA87B
:1069BC0041790904827912025118C0790818039997
:1069CC00491E88420AD993490818801C06E02D9963
:1069DC00685A401C6852FBF741F800208E49096840
:1069EC00599A91426F9A07D04A1C8B4B1A60132903
:1069FC0001DC00217391739A729288490968081816
:106A0C00CA0F89184910441AE00F2018471031207A
:106A1C00C0002F50A86F7390709EF0688021695849
:106A2C008822AA58401A504303F014FF00252A4626
:106A3C007B4B03F06FFD03F06BFE63218900744BFD
:106A4C00585076490C607399791A764A1160091A74
:106A5C007391754801600420305E7E21595E1F469B
:106A6C00401A03F0F7FE04460E469020385803F007
:106A7C00F1FE2246334605F04DFB2A46684B03F0E7
:106A8C0049FD03F045FE7399081A03F0E3FE2A460C
:106A9C00664B05F03FFB2A46654B05F03BFB5D9AC8
:106AAC00D3052A4605F036FB04460E4661480460C1
:106ABC0041609420385803F0CDFE2A465E4B03F01B
:106ACC0029FD2246334605F025FB02467390719151
:106ADC005A480260416006207099085E9821795EE0
:106AEC00401A03F0B7FE04460E46A420385803F0B3
:106AFC00B1FE2A46524B03F00DFD2246334605F0FB
:106B0C0009FB2A464F4B03F0BDFB739A719B05F0B2
:106B1C0001FB04460E46739500224B4B03F0B8FD67
:106B2C00002811D1002220463146484B03F0D0FDFD
:106B3C00002809D1002220463146394B05F0EAFAEB
:106B4C0003F0E6FD324A03E019200001304A1058E8
:106B5C00E421505072980028709D0BD0E869296A86
:106B6C00884201DDE8692862E869696A884201DACD
:106B7C00E86968620121364868910160354800680F
:106B8C00296E081ACD2149005052334E301D7C22FB
:106B9C00314605F03BF9314F381D39467C2205F062
:106BAC0035F9E869679030602869539038605998D6
:106BBC000546739E3746334607E0361D802E0D463C
:106BCC00719A1746729B20464AD02449739689596C
:106BDC00CC176140091BB9420C4600DC3C46719451
:106BEC00A94200DB29461C4A9259D4176240141B57
:106BFC009C42224600DC1A4672928442DDDB04463B
:106C0C00DBE7C046EC120000BC0E00201800005060
:106C1C0028000020FFFFFFFE780F00207C0F0020D3
:106C2C0000408F402C0F0020300F00200000084047
:106C3C00000049409005002080842E4188050020EA
:106C4C0065CDCD410000F03F00206140002061C0C7
:106C5C00040F0020640F0020A00C0020A00B0020CB
:106C6C00501AC1174840401A5190192801D30020DE
:106C7C006890181BC1174840441A074FF86D6821DB
:106C8C00795A03F0BDFE142103F092FE5094844215
:106C9C006F98024D05DB03E02800002001A00000E6
:106CAC006898002800D0B8E2074842688368981AB0
:106CBC00C1174840401A67992492511ACA1751407B
:106CCC00891A884203DC01E0A00C00200846044924
:106CDC00CC68E11ACA175140891A814203DC01E0E1
:106CEC00A00C0020014604480569281BC21750401F
:106CFC00801A884203DC01E0A00C002008460449FD
:106D0C004E69711BCA175140891A814203DC01E09C
:106D1C00A00C0020014604488769B81BC2175040DC
:106D2C00801A884203DC01E0A00C002008460549CB
:106D3C00C9694F91C91BCA175140891A814204DC99
:106D4C0002E0C046A00C002001460548026A4F989C
:106D5C004E92101AC2175040801A884203DC01E090
:106D6C00A00C0020084605494A6A4E994D92511ACA
:106D7C00CA175140891A814203DC01E0A00C0020A3
:106D8C0001460548826A4D984C92101AC217504021
:106D9C00801A884203DC01E0A00C0020084605495B
:106DAC00CA6A4C994992511ACA175140891A8142A0
:106DBC0003DC01E0A00C002001460548026B499859
:106DCC004892101AC2175040801A884203DC01E026
:106DDC00A00C0020084605494A6B48994792511A65
:106DEC00CA175140891A814203DC01E0A00C002033
:106DFC0001460548826B47984692101AC2175040BC
:106E0C00801A884203DC01E0A00C002008460549EA
:106E1C00CA6B46994592511ACA175140891A814238
:106E2C0003DC01E0A00C002001460548026C4598EB
:106E3C004492101AC2175040801A884203DC01E0B9
:106E4C00A00C0020084654900548426C4498101A37
:106E5C00C1174840411A54988142269103DC01E045
:106E6C00A00C0020014655910548806C4390801A77
:106E7C00C1174840411A55988142289103DC01E022
:106E8C00A00C0020014656910648C16C43984291D3
:106E9C00081AC1174840411A56988142299104DCBE
:106EAC0002E0C046A00C0020014657910648016D37
:106EBC0042984191081AC1174840411A579881428B
:106ECC002A9104DC02E0C046A00C002001465C9133
:106EDC000648416D41984091081AC1174840411A23
:106EEC005C9881422B9104DC02E0C046A00C00208F
:106EFC00014661910648816D40983F91081AC1176F
:106F0C004840411A619881422C9104DC02E0C04651
:106F1C00A00C0020014666910648C16D3F983E9139
:106F2C00081AC1174840411A669881422E9104DC18
:106F3C0002E0C046A00C0020014620976891FA4858
:106F4C00016E3E983D91081AC1174840411A689845
:106F5C0081422F9100DC01462F467191F248416E1F
:106F6C003D983C91081AC1174840411A71988142CA
:106F7C00309100DC014625467291EB48816E3C98BD
:106F8C003B91081AC1174840411A729881423191BD
:106F9C0000DC014673911F922196E348C26E3B9828
:106FAC00101AC1174840441A73988442329400DC7A
:106FBC0004462593DC48036F1E92991ACA17514058
:106FCC008E1AA642314600DC214633942395446F39
:106FDC001D93E21AD3175A40D31A8B421A4600DC7F
:106FEC000A462297856F1C942C1BE7177C40E41BE8
:106FFC009442274600DC1746C06F1B951A90401B25
:10700C00C5176840401BB842C84D00D905E19442F1
:10701C0000D902E18B4200D9FFE03398864200D9B7
:10702C00FBE073983299814200D9F6E0729831995D
:10703C00814200D9F1E071983099814200D9ECE09D
:10704C0068982F99814200D9E7E066982E99814281
:10705C0000D9E2E061982C99814200D9DDE05C987E
:10706C002B99814200D9D8E057982A99814200D9AE
:10707C00D3E056982999814200D9CEE055982899A9
:10708C00814200D9C9E054982699814200D8C4E0C5
:10709C00519803F0DFFB04460D46509803F0DAFBE1
:1070AC0002460B462046294603F034FA0022A04B38
:1070BC0005F030F803F02CFB15999E4B5852252007
:1070CC00C000185871903720C00073901A18679838
:1070DC00D0671698C00072901B185398D8672498E4
:1070EC00906795490D1DE0CD08694C6961948C69D8
:1070FC006694CC6967940C6A68949D67259D556766
:10710C005E67239D15671F67229DD566D8662198FB
:10711C009066619898668948719C046020985066C6
:10712C00669858664F981066679818664E98D065A2
:10713C006898D8654D989065486A8C6ACD6A0E6BD4
:10714C004F6B66978F6B6797CF6B68970F6C7197C8
:10715C0098654C9850655C65499810651D65489814
:10716C00D064DE644798906466989864469850643E
:10717C006798586445981064689818644498D0636C
:10718C00DF631F989063486C8C6CCD6C0E6D4F6DEB
:10719C0066978F6D6797CF6D68970F6E7197986331
:1071AC00439850635C63429810631D634198D062AE
:1071BC00DE6240989062669898623F985062679839
:1071CC0058623E981062689818623D98D061DF61F1
:1071DC003C989061486E8C6ECD6E0E6F4F6F6797BA
:1071EC008F6F6897C96F719198613B9850615C6122
:1071FC001E9810611D611D98D060DE604B4D1C986F
:10720C009060679898601B9850605F60494F1A981F
:10721C00739978507298719939500020FE49086022
:10722C00FE4E3768FE480068016840686A983C1A50
:10723C00601E84416D980028589800DC00207290E4
:10724C005B980140699881423A4A01D100F0C7FC31
:10725C00579161942520C1005058401C5C915050AE
:10726C005F98002816D1F14B181F006801044B9A47
:10727C001040189C2140081850401860F84C606968
:10728C00F849491C0204629B18400A401018294A0C
:10729C005840A061D06D010C6B9B1C0C22464A43DC
:1072AC009BB2594380B267934343689460430C0C80
:1072BC00090459185441030C0004401869906341A7
:1072CC00E94903C9014309D100204B218900194A1E
:1072DC005158E64A5143E44A1160506066937197E5
:1072EC00E34903C9014309D1002013210901114AC3
:1072FC005158DE4A5143DE4A11605060E4260D4F6E
:10730C00B85900281CD45220385A03F0EFFA002246
:10731C00D84B03F0FFF804460D46B85903F09AFA1F
:10732C0022462B463DE0C046A00C002001A00000E8
:10733C0000408F4028000020A00B0020640F00208C
:10734C00F86D6821795A03F05BFB0446B859614229
:10735C008842B85929DA03F07DFA73900D466A9188
:10736C00204603F077FA02460B460120C10769401C
:10737C00739803F0CFF856900D465020385A03F00E
:10738C00B5FA0022BB4B03F0C5F80022BA4B02F051
:10739C0079FF02460B465698294602F007FE739A6F
:1073AC006A9B04F0B7FE03F0B3F96A96709A906288
:1073BC0070205190385E916A081A9062D169D06938
:1073CC0000290FD4C117AA4E3268141875684D41A4
:1073DC00002320462946A54A03F04EFB1321090140
:1073EC00785018E04042C1179F4E326814187568E7
:1073FC004D410023204629469C4A03F03DFB4B217E
:10740C008900785078586C994843F96D03F0F8FA74
:10741C004F218900785234607560709CA06A616B52
:10742C00C217236B181820634A416263A06AE16F8C
:10743C00C217A36F1818A0674A41E267A06FE16FEB
:10744C0000256B9A2B4603F0FFFA2D21C9005491AD
:10745C007850606B216B699A511A669E3146814156
:10746C0004DAF8203A503846F830466036988001F5
:10747C00391849683858401EA9416A9C04DB05201C
:10748C0080013D5038184560F96D3498385AD8222F
:10749C007392BA5858235593FB5A9A4210DD4843BD
:1074AC0003F024FA2A46734B03F034F803F04AF93C
:1074BC003A59D317101A8B4102DA70480088451CD0
:1074CC006E4805805620385A29B2814228DD709CBE
:1074DC006663699820630020E067A067396E0A0C28
:1074EC00689E33465343679D6A4389B24D4371434B
:1074FC00160C1204AA185E410B0C0904891873416E
:10750C0017221201B950B9184B60649978506399DD
:10751C0048605B21890078506F99594A1170A065B9
:10752C00709E306B716B00256B9A2B4603F08CFAB6
:10753C00F06230693A99C9016691795A88425EDAEB
:10754C00739838586C99884259DD4E490888401C0C
:10755C00088080B20A2854D349480078002850D0BB
:10756C000A200880092040013958474A914242D9E3
:10757C003858464988423ED854997858002878584B
:10758C0000D5404270645B2080003958385800297F
:10759C0000D540423E49B064706C0028084623D4A4
:1075AC00432080003958F86D81426C981CD2F86DDC
:1075BC000028374818D05D98C0000A0C060C3746D6
:1075CC00574383B25A4388B243437043160C110499
:1075DC005A187E412F4F010C000480187141709E87
:1075EC00FA6D002303F048FA0599785200202449DB
:1075FC000870FBF7F3FF492080003D5001E0214863
:10760C00058064205690385A042800D9D8E005A18A
:10761C00085C40008744C046040F00202400002072
:10762C00900E00200C784D714000C04618000050A0
:10763C00F86D0023010C689D2A464A43679C614300
:10764C0080B2444368430E0C090461185641040C83
:10765C00000445187441F82038583946F83142E096
:10766C0000040050FFFFFF00A805002080EE36004C
:10767C00B0050020000059400000F0BF8E0F002024
:10768C00840F00208A0F00200F0E000080FC0A00DF
:10769C00FFFF00002800002011200201B85800282C
:1076AC0038DD432080003858549979580818C11790
:1076BC0035E0386E002800D182E00023010C689D73
:1076CC002A464A43679C614380B2444368430E0C8C
:1076DC00090461185641040C000445187441172024
:1076EC000101785879184968F44A03F049F92A4697
:1076FC00234603F0A9F9054662E05B208000395867
:10770C00002932D4002032E054997858002835D41E
:10771C00002035E0F86D5499795808180021336928
:10772C00669C3C5BB56C012D02DBBD58EA1701E091
:10773C003D6E002269921A19D30FD3185A10DB1719
:10774C0003F01EF900236C9A03F07EF9DB4E3246EF
:10775C00002303F015F92A46699B03F075F90546D9
:10776C00C0178543B5422ADA2AE038584042112125
:10777C0009017A58002A08DC3C6E0AE0785840422D
:10778C00432189007A58002A02DD7C58E11701E078
:10779C00FC6D00216991C1170026C84D2A4633465D
:1077AC0003F0EEF82246699B03F04EF96A1E33464D
:1077BC00B341121A8B4100DB2E1A002900D4354636
:1077CC0001204E9000023D50BD48026841681046B1
:1077DC00084308D10021179880003A58B948424311
:1077EC00B748026041604C92B74804684368204631
:1077FC0018436A9A08D100232720C0003C58B1488E
:10780C004443B148046043604D91B85800285093EC
:10781C004F940ED47220395AB8584843642103F05F
:10782C00C7F85F21890078505198385E7958081A4A
:10783C0001E0F02038585F21890078507A58D3172E
:10784C0073983858C11703F09BF800236C9A549323
:10785C0003F0FAF81722140153943D1969953A6E06
:10786C006B683E5986193E514B416B60639C636853
:10787C00649D7E59301878514B416360100C689BA5
:10788C0019464143679C604392B254435A43030CDC
:10789C00000426184B41100C110489195841699A9F
:1078AC005268539B1E46FB58CB1A0346934102DA8F
:1078BC00B95169994860639B58682A467959491EA1
:1078CC005499884101DBB9505960B8585968002562
:1078DC006B9C22462B4603F0B7F85B21890078504D
:1078EC00B8596999496822466995002303F0ACF8A8
:1078FC002F21C90078503798C000395838580029C2
:10790C000FD4C1174F9A1418509D4D410023204697
:10791C0029466C4A03F0B0F82721C90078506A4810
:10792C0017E04042C1174C9A14184D9D4D4100234D
:10793C0020462946634A03F09FF87099C866486E42
:10794C006C994843F96D03F05BF84F21890078522C
:10795C005B48046045607424385B0028B34900D14F
:10796C009AE1385B0128084602D0385B0846103093
:10797C0027990160385BAE4908807624385B002873
:10798C0000D1A3E1385B0128A849084602D0385B36
:10799C000846103062990160385BA64908805C98F3
:1079AC003858A54903F02CF8A4490968884204D03A
:1079BC00A24908600020FBF711FE5599785A7E5AAF
:1079CC00CF2149009E4D2C687C5202F08FFF9D4ABE
:1079DC009D4B04F09FFB02F09BFE73997F588742EE
:1079EC0002DD002028600EE0304602F07FFF974A4F
:1079FC00974B04F08FFB02F08BFE874200DBF4E127
:107A0C0000208F4908609349086093490A46934FB8
:107A1C00709E672080003A524F208000385A002810
:107A2C00084613D0F06E02F061FF04460D46306F2D
:107A3C0002F05CFF02460B462046294602F06AFD26
:107A4C000022874B04F066FB02F062FE8B2149009A
:107A5C0078528448006A84494843000C8349096879
:107A6C00401A164948438249096802F0A1FF81492E
:107A7C0040180A2102F09CFFCC22B8525A21785AA5
:107A8C00669BF852B85E6A243B5F984238DAB85A63
:107A9C00BB5E6C22BD5EAB4200DCB85ABA5E6E2394
:107AAC00FB5E3D5F95422C4610DC1446AA420FDA71
:107ABC007D5E944210D1002020E0C046A0860100DB
:107ACC009805002080EE3600A0050020AA42EFDBCE
:107ADC002A467D5E9442EED0AB421E4600DB2E461B
:107AEC009D4200DC1D46A11A0B467343AC1B00B231
:107AFC00801A6043C01802F05BFF709E6699785242
:107B0C005848C06958494843C117090C401800141B
:107B1C0056994143584808180A2102F049FFF08051
:107B2C000620315E359AB25E305E914202DDD02184
:107B3C00785205E0D221795E884201DAF0887081B2
:107B4C00484840695A9EB95B020C0B0C1C465443C6
:107B5C0089B24A4380B241435843130C12048A1829
:107B6C006341010C0004801859410B2273920023CD
:107B7C0002F006FF02F0C8FE0022404B02F0CAFCE5
:107B8C0002F0C6FD15210901785236488069B95BAF
:107B9C00020C0B0C1C46544389B24A4380B241433D
:107BAC005843130C12048A186341010C000480180A
:107BBC005941739A002302F0E3FE02F0A5FE002265
:107BCC002E4B02F0A7FC02F0A3FDA921490078522C
:107BDC00579869902A4E3A462A4D719F619C2A48C3
:107BEC006599405C518B002901D100F08DFC002877
:107BFC0001D000F089FC508B2449884200DDE5E07F
:107C0C00401E0A2800D9E5E24000C046784480882E
:107C1C004000874448023D002E022B02DF02A308DD
:107C2C001B0237020B021C019101C04618000050C8
:107C3C00860F0020820F002080510100380F002099
:107C4C00440F00207B14AE47E17AF03F0AD7A370B3
:107C5C003D0AEF3F3C0F0020FFFF000028000020F2
:107C6C0000005940E00E0020E40C0000280F00201A
:107C7C00240F002030750000A015FFFF00002441E8
:107C8C002400002001A00000B8050020F103000032
:107C9C00FAF78CFD00F035FCF84800880028F8490C
:107CAC0002D083204000395283204600B85B002864
:107CBC0003D0B85B884200D0EBE273983858B98E89
:107CCC00884200DBB7E00127FC48DAE2FC48008878
:107CDC000028F94902D04120800039524120860009
:107CEC00B85B002802D0B85B884239D173983858F9
:107CFC00398F8842F3482CDC6A9838583E21795EDB
:107D0C006C9A51438842F0480F994E9121DCCE2158
:107D1C00785E5E9ABA5E9042EC483A9A4E9218DCC3
:107D2C00CC22B85E5E9BFB5E9842E948529B4E9318
:107D3C000FDC785E6E99795E8842E64836994E91F2
:107D4C0007DBB85E6E99795E884209DA06204E90A0
:107D5C00E14801F0E3FD4E98B8536298DF490861A1
:107D6C00B85B002800D117E673983858798F884291
:107D7C0000DB11E66A9838583E21795E6C9A5143C3
:107D8C00884200DB08E6CE20395E4222BB5E994277
:107D9C0000DB01E6CC217B5EBA5E934200DBFBE5A7
:107DAC003A5E46203B5E9A4200DCF5E5795E385E31
:107DBC00814200DCF0E5B85B022800D1ECE5C84854
:107DCC0001F0ACFD0020B853C448E3E5C549884236
:107DDC0024DCC549884200D169E1C249884200D0FF
:107DEC00F8E16F9801F05EF88BE3C048006800285A
:107DFC00BF4A02D1BD480760384601460A318F425E
:107E0C00709E03DC0A38874200DBE5E1002010603D
:107E1C00B6490860109AB74FA749FAE5FD218900C9
:107E2C00884200D1A0E1B449884200D0D2E10120BF
:107E3C00FBF7D4FB65E36A9838581299795E6C9A13
:107E4C005143884200DBD5E10227AC4819E261942A
:107E5C00AB4802F0A1FEA7499C240859002800D188
:107E6C0002E2085902F0F6FC00252A467395A54B50
:107E7C0002F050FBA44A16687197576832463B468D
:107E8C0002F048FB0022A14B04F044F902F040FC44
:107E9C0094226A9297498850709AD0889823679355
:107EAC00C85290889A226892885299483246994EC4
:107EBC003B46904D719F02F06FFE285902F0CAFCB0
:107ECC00739C22468F4B02F025FB024692480B46D0
:107EDC0002F062FE6798285E904D02F0BBFC2246D1
:107EEC008F4B02F017FB02468E480B4602F054FEF5
:107EFC0068988049085E02F0ADFC2246884B02F07F
:107F0C0009FB024688480B4602F046FE6A987949FE
:107F1C00085802F09FFC22467C4B04F0FBF802460A
:107F2C0082480B4602F038FE814802F035FE2046AE
:107F3C00FBF754FB619CE4E27E48164602F02CFEF3
:107F4C006194CE24305BA0217052705E02F082FCF2
:107F5C000022734B02F0DEFA024677480B4602F021
:107F6C001BFE305F9821715E401A02F073FC739017
:107F7C006A9100226A4B02F0CDFA02466F480B461A
:107F8C0002F00AFE6E487197076846686D483A46DB
:107F9C00334602F001FE9C245648005902F05AFC6C
:107FAC000022584B02F0B6FA024667480B4602F024
:107FBC00F3FD5048005902F04DFC0022514B02F0E9
:107FCC00A9FA3A46719F3346524E02F0A3FA0022A8
:107FDC005E4B02F057F9739A6A9B02F09BFA0022EF
:107FEC005B4C234604F096F802F092FBA421414A24
:107FFC005050505802F02EFC00222346619C02F097
:10800C0089FA0022464B04F085F80022514B02F00D
:10801C0039F9024650480B4602F0BEFD4F4802F0BB
:10802C00BBFD00203D4DFBF7D9FA6AE2CC20105A7B
:10803C008C215052505E7E21515E411A4848006896
:10804C006C9A504302F0B4FC90212AE03120C0001D
:10805C00105890671346709AD0880A995852908895
:10806C007E215852D068802158501CE0FAF742FD0E
:10807C0047E20120FAF702FF43E2C046860F0020D8
:10808C00FFFF0000D42010588421505050588021FC
:10809C005158411A334800686C9A504302F088FCDE
:1080AC008821144A50500020FBF798FA29E200204E
:1080BC0000F0F8FE25E2C046FFFF0000EBCB000805
:1080CC00820F002024CE00080CCE0008E0C9000866
:1080DC002DCC000849C800080CCC00081800005032
:1080EC0002CA0008F3030000F20300003C0F00205A
:1080FC00440F002028000020D2040000F4CD00081A
:10810C00EEC8000800408F409005002080842E416E
:10811C0067CA0008240000206EC6000801A00000F9
:10812C00000059407DC6000800C9000800CD0008B9
:10813C000AC9000888C600089FC6000820C90008A4
:10814C0088050020AEC600082EC900080000F0BF4C
:10815C0065CDCD410000F03FE1C6000814CD00080C
:10816C00300F00202C0F0020FC4B196A186A1A697A
:10817C001A6900227592BB2278920622749205220B
:10818C0012067A920D9A120679923F220A401946EB
:10819C0076928002800E77905868002809D50846A0
:1081AC000838F54A0260F54A02604868002800D594
:1081BC00AEE048681199084200D1B2E0ED49081FC1
:1081CC00EF4A0260EF4A026048681199084200D0F9
:1081DC00A7E0A9E0EC4892E1EC4F6A983858519925
:1081EC00795E88420FDA00201060E9490860E9499D
:1081FC008A1E0EE4CE20395E4822BB5E99422BDDEE
:10820C000327E5483DE0601C1060E449884206D332
:10821C006A9838585199795A401A0899785208989E
:10822C00385E0128DE4C13DB5C983858DD4902F0CF
:10823C00E7FB216888420BD00899795EDA4D2A68F1
:10824C009309D21A51188A09029BFA5220602960AC
:10825C00D049699AFFF7DDFBCC217B5EBA5E934275
:10826C0007DD0427D1480CE0D14801F057FB619C95
:10827C0047E13A5E4C203B5E9A4200DB7AE30527ED
:10828C00CC4801F04BFBC14887530746CA48279995
:10829C000161B85B002801D1FFF76CFB739838586B
:1082AC00F98E884201DCFFF765FB6A983858129901
:1082BC00795E6C9A5143884201DCFFF75BFBCE2060
:1082CC00395E4A22BB5E994201DBFFF753FBCC219E
:1082DC007B5EBA5E934201DBFFF74CFB3A5E4E20AD
:1082EC003B5E9A4201DCFFF745FB795E385E8142CA
:1082FC0001DCFFF73FFBB85B022801D1FFF73AFB2B
:10830C00AE4801F00BFB0020B853AB48FFF730FB35
:10831C00AB4801F003FB974948681199084200D01B
:10832C004CE7A84801F0FAFAA74801F0F7FA74A84C
:10833C00F8F71AFC002864D0A44801F0EFFA306872
:10834C008C490968609A114223D03168091A6C9AD9
:10835C00914226D287490968609A114219D0316836
:10836C00091A6C9A91421CD282490968609A11428E
:10837C000FD03168091A6C9A914212D27D49096862
:10838C00609A114205D03168091A6C9A9142D7D380
:10839C0007E078490B688E4A521C0A608C490B42E4
:1083AC0006D074494868119A104348604868A8E0A0
:1083BC0070490968139A1142F3D03168091A6C9A02
:1083CC009142EED26B490968139A1142E9D0316897
:1083DC00091A6C9A9142E4D266490968139A1142BF
:1083EC00DFD03168091A6C9A9142DAD26149096876
:1083FC00139A1142D5D03168091A6C9A9142D7D38D
:10840C00CFE730685B490968609A114223D0316824
:10841C00091A6C9A914227D256490968609A1142FE
:10842C0019D03168091A6C9A91421DD251490968C8
:10843C00609A11420FD03168091A6C9A914213D28A
:10844C004C490968609A114205D03168091A6C9A36
:10845C009142D7D308E047490B685D4A521C0A6029
:10846C005B490B4200D1E1E16194424C6068119987
:10847C00084360606068574801F050FA3068216822
:10848C00619C609A114227D03168091A6C9A91420A
:10849C002BD238490968609A11421DD03168091AEB
:1084AC006C9A914221D233490968609A114213D0D7
:1084BC003168091A6C9A914217D22E490968609A50
:1084CC00114209D03168091A6C9A91420DD229498E
:1084DC000968609A1142D7D1264B19683C4C621C32
:1084EC001A602142619C00D1D0E122494868079A68
:1084FC00104348604868384801F010FA374801F0DA
:10850C000DFA002021494883729820406D9A121A66
:10851C00334800685E9908406D92104322D1306850
:10852C003168091A0A290BD83168091A0A2907D89F
:10853C003168091A0A2903D83168091A0B29EFD3B3
:10854C002748006840060BD46298F4306D905F9811
:10855C000028244E48D000204AE0C046102002409B
:10856C0000206D901F4E307D0028394647D1FDF715
:10857C0084FDC0461020024023016745AB89EFCD36
:10858C003B2A19087F6E5D4C60CD00082800002046
:10859C003C0F0020FFFF0000B0C90008312A00008A
:1085AC00400F002080510100480F0020CACB00086A
:1085BC0084CA000826C8000818000050D2C9000858
:1085CC0013C800088CC90008ACCD0008B5CB000856
:1085DC00FA830000BCCD0008A2C90008D4CD000865
:1085EC0010080050B80500204B98F749086001208E
:1085FC005F90307D0028394601D1FDF73EFD4A9849
:10860C00C00073903158052901D2FDF72DFD7197EB
:10861C002723F05C7290012037466A90C6438C1E6B
:10862C0026402837F74A02E0BF1CB61E73D0781ECE
:10863C00007850404208C0071AD06A405008D20750
:10864C0019D14208C0071AD06A405008D20719D174
:10865C004208C0071AD06A405008D20719D1450801
:10866C00C0071AD0E84845406A08E80718D119E055
:10867C005008D207E5D068404208C007E4D1500842
:10868C00D207E5D068404208C007E4D15008D207B1
:10869C00E5D068404508C007E4D16A08E80701D076
:1086AC00D94842403D7855406808EA0705D0D64D78
:1086BC0068404208C00704D104E0D34D4208C0070B
:1086CC0000D06A405008D20712D068404208C00758
:1086DC0011D15008D20712D068404208C00711D1FE
:1086EC005008D20712D068404208C0079CD010E056
:1086FC004208C007EDD06A405008D207ECD14208BE
:10870C00C007EDD06A405008D207ECD14208C00730
:10871C008AD06A4088E7C80705D1BC4E719F481CB7
:10872C002CD1FDF7A1FC08466A9DA843B74E301822
:10873C002525405D424090B24008B34DD20757D03A
:10874C006840719F4208C00756D15008D20757D0D5
:10875C0068404208C00756D15008D20757D068402D
:10876C004208C00756D15008D20757D0684042087B
:10877C00C00756D1481C01D1FDF776FC3019C05CFE
:10878C007118659BC95C09020818904201D0FDF76D
:10879C006BFC7298002806D09D48008B7299884219
:1087AC0001D0FDF761FC5F980028394601D0FDF738
:1087BC0064FC0E992831729B73548B208500002425
:1087CC0074510B98325C102A689500D1A2E0062AED
:1087DC0000D18BE0032A00D0A6E08D48008B002B43
:1087EC0000D1B8E0984200D1B5E00B228623FDE021
:1087FC00719F4208C007A8D06A405008D207A7D181
:10880C004208C007A8D06A405008D207A7D1420836
:10881C00C007A8D06A405008D207A7D14208C007A9
:10882C00A8D06A40481CA9D1FDF71EFC79490968FB
:10883C00139A114200D117E63168091A6C9A9142C9
:10884C0000D311E673490968139A114200D10BE663
:10885C003168091A6C9A914200D305E66D49096892
:10886C00139A114200D1FFE53168091A6C9A9142B2
:10887C0000D3F9E567490968139A114200D1F3E571
:10888C003168091A6C9A9142D0D3EDE561490968B7
:10889C00139A114200D128E63168091A6C9A914258
:1088AC0000D322E65B490968139A114200D11CE6F9
:1088BC003168091A6C9A914200D316E65549096839
:1088CC00139A114200D110E63168091A6C9A914240
:1088DC0000D30AE64F490968139A114200D104E605
:1088EC003168091A6C9A9142D0D3FEE54848008B46
:1088FC00002B01D0984213D134462734E378A27868
:10890C001002C018629DDB35A8423AD92520C00060
:10891C00414A57E03E48008B002B0CD098420AD0BD
:10892C002520C0003D4A4DE070186A9B8370099B5E
:10893C005A4042705DE03246273257791079000276
:10894C00C31918467C387B24E443A0422AD825203E
:10895C00C000392235E032462732567910790002B0
:10896C00801905467E3D0A9BDF438323BD422DD2F1
:10897C0003223AE0795E385E814200DB89E4062707
:10898C0070E44000224F3D1826796E7064793C5497
:10899C001E484018447106711C4EC3708270062428
:1089AC00447027E07297D5789478200242199F186A
:1089BC001B4BD819401E984200D352E12520C00011
:1089CC00069A1201325214E018000050D5789778AC
:1089DC003A02729552198518669511484019401E35
:1089EC000F4DA84200D37AE10222084E7018827013
:1089FC004370032425466A98854372182E46014F0E
:108A0C0014E0C046FFFF000001A00000B8050020E4
:108A1C00280000201020024086020000860B000077
:108A2C0024FEFFFF921CB61E00D181E013787B4020
:108A3C005808DB071DD0DA4B58404308C0071BD140
:108A4C005808DB071DD0D64B58404308C0071BD134
:108A5C005808DB071DD0D24B58404308C0071BD128
:108A6C005808DB071DD0CE4B58404308C0071BD11C
:108A7C001CE04308C007E3D0C94843405808DB0753
:108A8C00E1D14308C007E3D0C54843405808DB0791
:108A9C00E1D14308C007E3D0C14843405808DB0785
:108AAC00E1D14308C00701D0F848434057785F40F4
:108ABC007808FB071DD0F54B58404308C0071BD165
:108ACC005808DB071DD0F14B58404308C0071BD199
:108ADC005808DB071DD0ED4B58404308C0071BD18D
:108AEC005808DB071DD0E94B58404708C00799D000
:108AFC001BE04308C007E3D0E44843405808DB07B9
:108B0C00E1D14308C007E3D0E04843405808DB07F5
:108B1C00E1D14308C007E3D0DC4843405808DB07E9
:108B2C00E1D14708C00700D17CE7D848474079E736
:108B3C00E00703D13A0AD44B689D3DE0D24B58195B
:108B4C00405C4740B8B24008D04DFA0719D0684095
:108B5C004208C00718D15008D20719D06840420803
:108B6C00C00718D15008D20719D068404208C00776
:108B7C0018D15008D20719D068404708C00718D13F
:108B8C0018E04208C007E6D06A405008D207E5D189
:108B9C004208C007E6D06A405008D207E5D1420827
:108BAC00C007E6D06A405008D207E5D14708C00795
:108BBC0000D06F40689D3A0A18194754401842700B
:108BCC000C20659A9854A41C5C51A2B2504250419E
:108BDC001A6813467C335D68202D6F9D00D10546C5
:108BEC00002D719F34D196680C98864202D1106981
:108BFC0000282DD0187801282AD0104654304480F3
:108C0C00DD600480A0484018106537985860506E9D
:108C1C00019988420DD10C98864203D11069002825
:108C2C009E4800D09E481D7010671168083103984B
:108C3C000BE00C98864203D110690028954800D0AF
:108C4C0095481D701067116809980A6802430A60FC
:108C5C0000208D49739A8850087539468B4DFDF765
:108C6C000CFA61956800669463021818854B1D1800
:108C7C000026AC19844883192E20185C60702F20B4
:108C8C00185CA855501CB8421BD23020185CE07000
:108C9C003120185CA070901CB84212D23220185CA3
:108CAC0060710498185C2071D01CB84209D2342031
:108CBC00185CE0713520185CA0710836121DBA42A0
:108CCC00D7D3714E7018729A427100220271619A58
:108CDC00C270669A82701022427006248AE66A4D2F
:108CEC00681873002E4683700323437072984000FB
:108CFC007B021818634B18187290669D6791301997
:108D0C0072990B195F789526760087558719085D3F
:108D1C007870501CA84219D2D878B8709878F8702E
:108D2C00901CA84214D25879387118797871D01CDB
:108D3C00A842554E67990FD2D879B8719879F871C5
:108D4C000834121DAA42DAD3E41C53E6641D00E079
:108D5C00E41D4D4E67994DE609344BE6BFF34F8F3A
:108D6C00444914394A480860BFF34F8F00BFFDE7F0
:108D7C0030682168C90701D0FDF786F8A168C907DA
:108D8C0005D1A1683D4A1140589A1143A160316840
:108D9C00091A0329EDD32168C907EAD1FDF737F881
:108DAC0001A000000A68A568344B1D400346589882
:108DBC000543A560579802409A18D2082369119D63
:108DCC00AB4229D25B9883042D4D2D681D40AB0C12
:108DDC00072B21D3DB1E589D9D407B957B9B5B080D
:108DEC007B937B9B002B17D07B9B5B1E7B937B9B8E
:108DFC00002B11D07B9B5B1E7B937B9B002B0BD0A2
:108E0C007B9B5B1E7B937B9B002B05D07B9B5B1E14
:108E1C007B937B9B002BE7D10B68579883431343C1
:108E2C000B60A168154A11400F9A1143A16031687B
:108E3C00A268D20712D03268521A032AF8D3A26859
:108E4C00D207F5D00C4A906D102101439165D06D7D
:108E5C0058990843D065D05DFCF7B1FFE168729872
:108E6C000143E1600448806D589908430F99884389
:108E7C00FCF704FE20ED00E0840D0020E8FFFF7FEE
:108E8C000827014028000020B805002001A00000A0
:108E9C000400FA05B11300085BC400085513000860
:048EAC0033C00008C7
:108EB000F0B589B00021069103910291F14C216A2D
:108EC0003F220A400492216A8902890E0591256990
:108ED000ED49079122690A40089200284DD0EB48DD
:108EE00000F022FDE8B2AA2800D08DE0BB20069059
:108EF00002200290606800280BD520460838F84907
:108F00000160F84901606068002802D5F64800F069
:108F10000BFD0126B5076068400007D5201FF44906
:108F20000160F44901606068284202D0FA4800F00C
:108F3000FBFC0195FA4800F0F7FC02A8F7F71AFECF
:108F40003704002864D0F74800F0EEFCEB480168D5
:108F500022683A4200D0B1E02268E94B5D1C2560EE
:108F60001A4203D12268520300D5E5E060680199F6
:108F700008436060606809B0F0BDE8B2AA2800D17B
:108F8000D6E0CC2800D1D3E0AA200690022002909F
:108F90006068002809D520460838D1490160D149C8
:108FA00001606068002800D5C4E0D04800F0BCFC37
:108FB000606840002AD50126B507201FCC49016012
:108FC000CC4901606068284220D1CB4800F0ACFC5D
:108FD00002A8F7F7CFFD002800D1D4E0C748016808
:108FE0002268D20300D525E12268C54B5F1C2760AB
:108FF0001A4203D12268520300D549E16068284330
:1090000060606068BF4891E0C4488FE0C2488DE06E
:109010000096BA4E7D2130682268CD003A42B84BA6
:109020002FD121685A1C2260194203D121684903BB
:1090300000D5B7E060680199084360606068B34894
:1090400000F072FCAE4B3068216839425CD0316868
:10905000091AA94260D22168394255D03168091AEB
:10906000A94259D2216839424ED03168091AA94221
:1090700052D22168394247D03168091AA942E3D354
:109080004AE03168091AA942D4D221683942C8D0CD
:109090003168091AA942CDD221683942C1D031685C
:1090A000091AA942C6D221683942BAD03168091AD0
:1090B000A942BFD221683942E3D1B2E77D22D20072
:1090C00003685B1A934200D350E723683B4200D108
:1090D00042E703685B1A934200D347E723683B42A9
:1090E00000D139E703685B1A934200D33EE7236857
:1090F0003B4200D130E703685B1A934200D335E767
:1091000023683B42DCD127E721685A1C22601942C0
:1091100002D1216849036BD40098C00761680143FC
:10912000616060687A4800F0FFFB7F4800F0FCFB5C
:1091300009B0F0BD6C48F9E7B2047D23DB00056897
:109140006D1A9D4200D311E72568154200D10DE745
:1091500005686D1A9D4200D308E72568154200D1C5
:1091600004E705686D1A9D4200D3FFE625681542A5
:1091700000D1FBE605686D1A9D4200D3F6E625682E
:109180001542DCD1F2E6604800F0CEFBF7F7ACFB0D
:109190005E4800F0C9FBF7F749FB5D4800F0C4FBEF
:1091A0005C48C3E7009989043268121AAA4200D3C6
:1091B00040E722680A4200D13CE73268121AAA420C
:1091C00000D337E722680A4200D133E73268121A27
:1091D000AA4200D32EE722680A4200D12AE7326869
:1091E000121AAA4200D325E722680A42DCD121E7FD
:1091F000009989043268121AAA428DD222680A4262
:109200008AD03268121AAA4286D222680A4283D0D1
:109210003268121AAA4200D37EE722680A4200D1BD
:109220007AE73268121AAA4200D375E722680A4226
:10923000E0D171E732047D23DB0007687F1A9F428B
:1092400000D3DBE62768174200D1CDE607687F1A16
:109250009F4200D3D2E62768174200D1C4E60768D0
:109260007F1A9F4200D3C9E62768174200D1BBE6A8
:1092700007687F1A9F4200D3C0E627681742DCD1F7
:10928000B2E6C0461020024000604F078CCD0008B7
:10929000B2047D23DB000668761A9E4200D3ADE659
:1092A0002668164200D1A9E60668761A9E4200D3C7
:1092B000A4E62668164200D1A0E60668761A9E4209
:1092C00000D39BE62668164200D197E60668761A18
:1092D0009E4200D392E626681642DCD18EE6C04656
:1092E00023016745AB89EFCD13C800087AC9000890
:1092F0003B2A19087F6E5D4C41CB000824000020FA
:10930000FA83000077CB000870CD0008BCCD0008C0
:10931000A2C9000856CB00088CC9000898CB0008E9
:0C932000ACCD0008B5CB0008D4CD00088F
:10932C000C490868401C08600B480268521C02601B
:10933C00D2087D2A0CD30968084A914208D30849FF
:10934C00CA6D521CCA6500220260886D401C88657B
:10935C007047C04624000020340F0020214E00002E
:04936C00F0000020ED
:10937000F0B583B03748001F0568374A1468206885
:1093800004260190304041424141106C1C230340AF
:1093900037469F40384602952840424242410A43A0
:1093A00030D0009401200226019D2A4632405142CD
:1093B00051419E40029A1642074600D00F46002FA8
:1093C00032D008210D4069426941DA40120700D5C8
:1093D0000846002826D1242000211F4C2154009A41
:1093E00010680E2188431060012001469940194BF6
:1093F0001A680A431A60E06325216054616B0029F2
:109400000ED10FE02068800602D42068B0432060AF
:1094100010490868384308600F48016B002901D0E3
:109420000D48884703B0F0BD2346206880060A4AED
:1094300006D418680A218843186025200121115498
:10944000242017540349086830430860D16A002972
:0C945000E6D1E7E704000240E80D002030
:10945C00F0B58AB098480168C8690A6809924A68E8
:10946C0001220792120706928A68089204074FD0CD
:10947C00069A531C089A134001252A0216462036D8
:10948C00099F3E401E4343D03A4056425641C207C4
:10949C00079A00D03246002A05D10D628822864FE9
:1094AC00BE582E43BE50089A15406A426A41860740
:1094BC00079E00D51646002E08D102220A62882289
:1094CC007D4EB658042737437B4EB7506A426A41EB
:1094DC004507079D04D4002D04D0002C0CD417E0B4
:1094EC001500FAD104220A628822734FBD58022655
:1094FC002E43BE50002C0BD52022099C2240134336
:10950C0006D008220A6288236B4DEC581443EC50A9
:10951C000125EA050492020513D5089A049B1A400A
:10952C00AB06099C23409A180BD0EA020A628422EB
:10953C002023614CA3508022A350604A1575604BC8
:10954C00D554202203460592134003931CD0089A4D
:10955C00069B1A40099B059C2340134314D04522BB
:10956C00D200564B9C588426534FBE59222E30D1D4
:10957C002E02B4422DD21C194E6A2727E655504CA8
:10958C001D559C58641C9C50802306461E403DD0A3
:10959C00089A049C2240099C1C40144336D0474A2C
:1095AC001268D458212C1DD1174656373C88002CF4
:1095BC00146802941FD0146D019424780097029FB4
:1095CC00BC62019C641C1465009C2288521E228083
:1095DC0018E08A69082313438B61802306461E40DA
:1095EC00D6D113E0126814689C43146014684027A9
:1095FC002743176006E022689A43226022684027BE
:10960C0017432760232212012C4CA55402954027A6
:10961C00099C3C4062426241400600D50792079883
:10962C0000280CD10868B8430860234D0598E85011
:10963C00244800220270842022242C502A6788227D
:10964C001D48805800282BD0842022241A4D0790C6
:10965C002C500398002809D0089D039106992940A5
:10966C00099D059805400D4303991BD1002E17D079
:10967C00089D049A1540099A1A402A4310D00A688A
:10968C00BA430A600C4D0598E85007982C502620D8
:10969C000A4900220A5423200001029B0B542A671A
:1096AC000AB0F0BD8869082303438B61002002498E
:1096BC0088500AB0F0BDC046940A0020B8050020BE
:0896CC0031020000DE05002060
:1096D40001204102074A13689B0503D453680B42D7
:1096E40004D17047116053680B42FAD051600249AB
:0C96F400086070470C180240040F0020B2
:10970000F0B583B05D4C2068C5680226294631401B
:109710004A424A410769394631404B424B41134363
:109720002346574A0ED11146FE31016101211977B6
:109730008069800704D05148F8F722F9504A23463F
:109740000020187701240420294601900140484256
:1097500048417907214600D50146032000020290C6
:10976000002910D118681146FC3101611E7780690B
:109770000299084205D041481E46F8F701F9404ACF
:109780003346002018770826294631404842484190
:109790003907214600D5014600290FD11868114626
:1097A000F831016101991977C069800704D0334805
:1097B000F8F7E6F8324A314B00201877102129409B
:1097C00048424841F906214600D50146002910D1FA
:1097D00018681146F03101611E77C069029908428C
:1097E00005D026481E46F8F7CBF8254A3346002018
:1097F00018770121294048424841F907214600D005
:109800000146002903D118681146FF31016180200B
:109810002840414241414122D2011742224600D014
:109820000A46002A02D11968164A0A61414241419A
:10983000F805204600D508460028114A01D11868CD
:10984000026140212940484248417906214600D51D
:109850000146002903D118681146C031016120205A
:10986000054068426841B90601D403B0F0BD040068
:10987000FBD11868E032026103B0F0BD440E002055
:08988000FFFEFFFF7FDFFFFF89
:10988800B0B51E4D2C1F20688006400F411E0329CD
:1098980022D81B487944097949008F442301171AB3
:1098A800296803220A40032A00D016482968490675
:1098B800490F491C01F0A6F829684904490E484394
:1098C8002968490F491C01F09DF80BE07D20000232
:1098D80008E00120C00305E00C3D28688004410F22
:1098E8000848C84008490860226892093C23134088
:1098F800064AD258D0400860B0BDC0460C1002409D
:1099080000127A000024F40020000020C4BE0008E1
:1099180080B50249096802F0E2FD80BD140000200C
:10992800B0B5044608480568204602F09DF902468D
:109938002846214602F000FD401C03D00A20FFF70C
:0C994800E7FFB0BDC043B0BD140000201C
:10995400C20F490089184000034A40428A4101D39A
:0C99640000207047012070470000E0FF69
:109970000122D2079143034A4A40104341424841E1
:089980007047C0460000F07FB3
:10998800074A0A40531E9A41C00F49000818054962
:10999800884201D300207047012010407047C0461C
:0899A8000000F07F0000E0FF69
:1099B00030B50E4B5D1C0C0D2C4011D0AC420FD0BD
:1099C000A2189A4206DD0120C00701400948091883
:1099D000002030BD002A04DD054B1940120511435B
:1099E00030BD0120C0070140002030BDFE0700004F
:0899F000FFFF0F800000F07F73
:1099F80010B54B005B0D084CA34201D0002B02D1DF
:109A08000023136010BD054C1B191360044A114054
:109A1800044A891810BDC046FF07000002FCFFFF7A
:089A2800FFFF0F800000E03F8A
:109A3000F0B587B00025EC43584E0494671C3446BB
:109A400000956C415D0003956D0D554D059577D0E2
:109A50000297C50F06914F0001977F1945000499A1
:109A60004D1BBE416CD3D50F03994D195600029979
:109A70008E1BAC4164D30125EC0706990C4005947C
:109A8000484C0E4626402340141A1C46B44175D259
:109A90002C05019F7F0D0494039505D02546641E77
:109AA0000E4626402E430BE0A64209D2E904344676
:109AB000C50F6600761940007F1E8C423446F7D3EE
:109AC000190D394C214006D0049D6C1E23402B43B8
:109AD0008F4221DC2AE004998B4210D20399C904F9
:109AE000069100211C46D30F6500EB185200491E59
:109AF000069DAC421C46F6D38F420DDC16E00021D9
:109B0000002F09DC12E005463446E80F64002618F1
:109B100068007F1E8F4208DD851A34469C41F2D4CE
:109B200050405E400643F0D10AE00F460546A81AB1
:109B300031469941049C05D455405E402E4303D1E3
:109B4000009818E02846314621420AD1039DEA04D4
:109B5000C30F4C00E31840007F1E11421946F7D096
:109B600001E00B46039D002F11DD791E059A9A181E
:109B7000090551180591059907B0F0BD42405E40B6
:109B8000164300D00591002EF5D10020F3E7EA1B23
:109B900000F0DCFE0B460021E8E7C046FFFFDFFFD8
:0C9BA0000000F87FFFFFFF7FFF070000C0
:109BAC00F0B583B00C462A494B1C220D1A40531EAB
:109BBC008B4242D228498A4206D20020002C014610
:109BCC0039DA284903B0F0BD33318A4202D9214633
:109BDC0003B0F0BD1F495518029021462A4600F0EB
:109BEC009FFE1E4A11400143484248410027002C69
:109BFC0001DA394600E00121014301911849384648
:109C0C002A4600F0ADFE2A4605460E46264002982E
:109C1C000540F843401C1149794100F091FE0A4679
:109C2C003146019C2B187241002C00D11146002C9E
:109C3C0000D11D46284603B0F0BD002A02D10121F7
:109C4C00C9070C402146002AF5D1002003B0F0BD15
:109C5C00FE07000001FCFFFFFF030000FFFF0F00E9
:089C6C000000F0FF0000F0BF52
:109C7400F0B587B00A0D521E494B9A4212D206AA79
:109C8400FFF7B8FE4B4A821A494A0B469341069C99
:109C94001CDA0022494B00F0F9FA641E05940446CC
:109CA4000D461EE0C30F4A00D318440064423D4CE5
:109CB4009C416FD3520D6FD000290A4600DA3B4A0B
:109CC400002900DA0020114607B0F0BD00223A4B0B
:109CD40005460E4600F0DAFA0594044628460D4679
:109CE40031460026F2430496FFF760FE344B00220F
:109CF40000F0CCFA02460B462046294600F00EFC42
:109D040003900F4602460B4602F008FA04460D463D
:109D14002C4E0221304622462B4602F010FC2A4AE1
:109D24002A4B00F0B3FA0290019110360321304619
:109D340022462B4602F02BFC02460B460298019960
:109D440000F0ECFB22462B4602F0E8F9039C224685
:109D54003B4602F0E3F922463B4600F097FA0646FA
:109D64000F46059800F07AFD04460D46184A194B33
:109D740002F0D4F932463B4600F088FA06460F4614
:109D8400154B20462946049A02F0C8F932463B4650
:109D940000F07CFA07B0F0BD0349002007B0F0BD25
:109DA400FE0700000000E0FF0000F0FF0000F87F65
:109DB4009EA0E63FCE3B7F660000F0BF0000E0BF00
:109DC4000000E03FC00000089AB5B312FF0750C07E
:0C9DD400A80C615C10D02BBF0030E63FF3
:109DE000F0B585B05B4A531C0C0D1C40631E9342BA
:109DF00000D393E05B4A121A594A8A4100DAA7E07D
:109E000000235A4A121A584A8A411A4600D281E05F
:109E10000122D2070B469343574A821A554A93416F
:109E200076D3564A564B02900D4602F079F901223C
:109E3000D2072A40534BD31800242246049400F042
:109E400027FA00F06BFC039000F00AFD06460F466F
:109E50004D4B002202F064F9029A2B4600F018FAEA
:109E600004460D46494A4A4B3046394602F058F9F5
:109E700022462B4600F00CFA06460D4602460B46DB
:109E800002F04EF90746434A434B0C46029102F05A
:109E900047F9424A424B00F0FBF93A46234602F0AA
:109EA0003FF9404B049C224600F0F2F932462B4623
:109EB00002F036F905460E46204632492A46334618
:109EC00000F0CAFA01900091374A384B3846029C9C
:109ED000214602F025F9364A364B00F0D9F93A46C8
:109EE000234602F01DF9019A009B00F0D1F90246C9
:109EF0000B462846314600F013FB049A214B00F034
:109F0000C7F9039A521CFFF753FD03460A4601E0C6
:109F1000174A00231846114605B0F0BDC20F4B008A
:109F20009A1843005B420C4B9341EED30122D207B7
:109F30000B469343094A5A40024300D071E7002977
:109F40000A4600DA0022002900DA00200346E1E791
:109F5000024ADEE7FE0700000000E0FF0000F07F9D
:109F6000422E8640EF39FAFE2B2386C0D2BC7ADD22
:109F70000000F03FA19CC73B2342920C3CF92F9E6E
:109F80002C15F73F0000E03F0030E6BFA80C615CF5
:109F900010D02B3F1CDC586FA452F13EE0F6B36F9B
:109FA000E4707C3F0000D03F0938DE6F993F403FAE
:089FB000B35142718E71AC3F08
:109FB800F0B587B01E460B4604460020C743924DB5
:109FC800791C2946414159400294214300D1A9E016
:109FD8007400610D8D4900D112E103970495069232
:109FE8008C4F7A1E05935D006B0D5B1E934273D2F6
:109FF800320D3A40884BD218521E9A426CD30698BA
:10A00800314600F087FB074600F026FC0122049247
:10A01800D407A742059D32D0069A504071400143AB
:10A028002DD1002F019745D0F81747403E1A774F9A
:10A038000024039402980BE04242224006983946D5
:10A0480002F06AF804460F4676082846059D33D084
:10A05800012E039A00D002460694012E6B4B00D0C5
:10A068002B460446294602F057F82A46054605912C
:10A07800304604990840654BDED01346DCE7049669
:10A088000022029E304629462F46134600F022FB46
:10A09800002803D06549002007B0F0BDA74330462B
:10A0A8003946FFF7E3FD069A049B02F035F8FFF7FF
:10A0B80093FEA5E0554F00240020544922463B4614
:10A0C80000F02AFA019A002A00D43946002A00D55D
:10A0D80096E0204607B0F0BD3746029EF20FAA1858
:10A0E80073005B1E4E4B534120D20125069EF20F92
:10A0F800A21873005B1B494B9A411BD2444A059B2B
:10A1080013421BD0474C1A466240029E324332D05B
:10A118001A463F4B5A40324348D1002F5BDA01467A
:10A1280007B0F0BD2046194607B0F0BD3046059986
:10A1380007B0F0BD3046394607B0F0BD30463E4660
:10A148000446394600F0E6FA074600F085FB324639
:10A158004A4023464340134300D057E70021002ECE
:10A16800084600DA2A49FA074AD0EA07059B13404D
:10A17800591807B0F0BD0490002F00DB2448059063
:10A18800069C20463E46394600F0C4FA074600F0D1
:10A1980063FB714060400843059802D1E8070599C0
:10A1A8000818F90700D005900498C0E76740069A98
:10A1B8003A4313D11C4A059B5A40334632431FD0B9
:10A1C800E807059A824300211846039B181A049849
:10A1D8009041084614D30E4907B0F0BDE807059929
:10A1E80081430020039B9A1B049A8A41014607D2A7
:10A1F8000D48059941403046084303D004494AE7D1
:10A2080007B0F0BD014946E7FFFFEF3F0000F03F10
:10A218000000F07FFF07000002F8FFFF0000E0FFEA
:10A22800FFFF1F000000F0FF0000F0BF0000F87FF4
:10A2380070B5040011D0E017214641400D1A1049AD
:10A248000020104E02E008366D0807D0EA07FAD061
:10A258000CCE083E01F060FFF5E70949084E0246BA
:10A2680000200B46314616461D4600F055F9002CD5
:10A2780001D502D570BD3046FCD4294670BDC04614
:08A288000000F03FE8000008AF
:10A29000F0B40125ED070F005F405AD48B4200D186
:10A2A000824205D950404240504059404B405940AD
:10A2B0004E18760DDF187F0D3BD0741C640529D035
:10A2C000F41B352C26D80E0DDB022B43DB0AC9020A
:10A2D0002943C9121700202C1ED2E741E240574003
:10A2E000E3415A40A340E3405A40002480185941BA
:10A2F0000AD3B21C520521D0C207012F62411700B8
:10A300004008CB0718434908013636054208AF41DB
:10A3100060417141F0BC7047203C06D01F00E7410E
:10A32000E3405F400024012A6741C0186141EBD33C
:10A33000DFE7002EEED129400020EBE701363105A2
:10A340000020E7E7E742E5D10020C143090DC90439
:10A35000E0E76B400E00871A9E4104D26E40C01B9E
:10A36000B141D21973414E18DF18AC0AE642E9D266
:10A37000760D7F0D31D0F41B362CCBD8B4460E0DA4
:10A38000DB022B43DB0AC9022943C90A012C32D85C
:10A3900004D1D4075208DF073A435B08EF0A64424E
:10A3A000904199411ED0002239424DD1241940419B
:10A3B00049410124394204D101340018494139424C
:10A3C000FAD06246A24204D9361B013E36058919ED
:10A3D000A0E7F10AC90700209CE736429AD1002085
:10A3E000002197E70200224394D0B842DED2010058
:10A3F00020002024E3D1202C13DD203CE241170073
:10A40000A240E2405740E3415A40A340E3405A4053
:10A41000012FBF410137174300227C4298419141EF
:10A420000CE01700E741E2405740E3415A40A340A7
:10A43000E3405A407C429041994100220F0303D2ED
:10A44000013E241940414941013E36054708AC41CF
:08A4500050417141F0BC70475E
:10A45800F0B40125ED076B40004C204797A2000897
:10A4680030B405004D400124E407254042004B006C
:10A47800120E32D01B0E3CD0FF2A33D0FF2B3FD018
:10A48800D21800022043000A09022143090AC4B273
:10A498004C43000AC3B24B43000A4843210A5B18E5
:10A4A800190A091801D44900013A080A7F3A2ADB37
:10A4B800FE2A0FD2D2051C43240601D001242143D1
:10A4C800C9B280295041802901D140084000284361
:10A4D80030BC7047FF20C005F9E71B0EFF2B0AD0E0
:10A4E8002800F5E7400206D1FF2BF3D1490202D13B
:10A4F800F0E7FF2AF4D17F2000010C300005E7E7E0
:10A508004902F8D1E6E743020132E9D15B1202338E
:08A51800E6D9D805E4E7C046CE
:10A52000F0B40125ED070C005C402C40A446AE0AB7
:10A530004C18DF18F4423DD2F74245D2640D4CD09E
:10A540007F0D3CD0E41BC9022943CF0ADB022B4319
:10A55000DB0A0600B61A9F4104D2013CB6197F41BE
:10A56000B6185F416812800D241838DD0018844247
:10A5700025D8E80C0021B6197F41B61A9F4103D3B4
:10A5800040414941F7D304E0B6185F410018494102
:10A59000F1D32405B6197F41B61A9F4105D337433D
:10A5A000C20717430022012F504161416246114307
:10A5B000F0BC70470CD100280AD1F74208D2002025
:10A5C000C143490D0905F1E7002A01D1F74206D040
:10A5D0000020C143090DC904EAE77F0DF8D000202F
:04A5E0006146E5E704
:10A5E40030B401256D054C00E54215D85C00E54208
:10A5F40012D80C001C436400044314430FD005D24A
:10A6040082428B418041013030BC70479042994175
:10A614008041013030BC7047002030BC70470120BD
:04A6240030BC70478F
:10A6280070B4012676054C005D00E6420CD8EE4277
:10A638000AD825430543154303D0994204D19042D3
:10A6480002D1012070BC7047002070BC7047C04622
:10A6580030B401256D054C00E54215D85C00E54293
:10A6680012D80C001C436400044314430FD005D2D5
:10A67800904299418041013030BC704782428B4101
:10A688008041013030BC7047002030BC7047012049
:04A6980030BC70471B
:10A69C0030B401256D054C00E54215D85C00E5424F
:10A6AC0012D80C001C436400044314430CD005D294
:10A6BC0082428B418041404230BC7047904299416C
:10A6CC008041404230BC7047002030BC7047C046CF
:10A6DC0030B401256D054C00E54215D85C00E5420F
:10A6EC0012D80C001C436400044314430CD005D254
:10A6FC00904299418041404230BC704782428B412C
:10A70C008041404230BC7047002030BC7047C0468E
:10A71C00F4464A1805D200F063F801D5C01740087A
:10A72C00604701235B05D34206D200F059F801D5EE
:10A73C000120C0074042604701D10042F5D0D0173C
:04A74C00400870470A
:10A750004A00520D01239B02D21A01321DD45242EB
:10A760003F321DDD8C46C902430D1943C00201234F
:10A77000DB071943202A02D308000021203AD141E7
:10A78000D04048409140D140484063461B4203D5E9
:10A79000002340428B411900704700200021704780
:10A7A000002801D0012211434B0001225205D3425F
:10A7B00000D959080020C90FC90701D4C043410876
:04A7C0007047C046D8
:10A7C40041000DD2090E7F390AD449421F3105D404
:10A7D40000020122D2071043C8407047C8177047CF
:04A7E400002070479A
:10A7E8004A0010D2520D03231B02FF33D21A0AD497
:10A7F80052421F3209D4400DC90208430123DB0726
:10A808001843D040704700207047D0177047C046A3
:10A818004B001BD25A0D01239B02D21A013215D4C8
:10A8280052423F3215DBC902430D1943C0020123CE
:10A83800DB071943202A02D308000021203AD1411E
:10A84800D04048409140D140484070470020002106
:08A858007047D01701007047A2
:10A86000054B004206D5404200B5984708BC01227E
:0CA87000D207114318470000F9A80008A7
:10A87C000B00034329D0CA0FD200043212023D321E
:10A88C00094203D5002349424042994102D10100BB
:10A89C000020203A0B0C04D1103A0904030C194384
:10A8AC000004094203D4013A00184941FBD58446FF
:10A8BC00C00A4B051843C90A120563465B055B4188
:0CA8CC0002D3012B00235841514170477A
:10A8D8009D2201000AD002D4013A4900FCD5D205D4
:10A8E800080A0906494100D3012950417047C0466A
:10A8F80042221201033A010007D002D4013A00189B
:0CA90800FCD51205C30A400599187047E1
:10A914000B00034305D0042212023D320942014BCD
:08A924001847704799A80008CC
:10A92C00202A07D203009040914052422032D3405B
:10A93C0019437047203A0100914000207047C046EF
:10A94C00202A07D2D0400B00D140524220329340F3
:10A95C0018437047203A0800D04000217047C04689
:10A96C00202A07D2D0400B00114152422032934092
:10A97C0018437047203A08001041C9177047C04669
:10A98C0030B5514343435C18010C130C0D005D436F
:10A99C00641992B2514380B242430D0C090452180F
:10A9AC0065415843010C00048018694130BDC04614
:10A9BC00CA1751408B1A17D0C1174A4094464840C9
:10A9CC00411A48081A0000E052008242FCD90020CB
:10A9DC0000E05208914200D3891A40419A42F8D1C2
:10A9EC0062465040801A704710B500F095F810BDC3
:10A9FC0007B5FFF7DDFF0EBC4243891A00BDC04608
:10AA0C000A0015D00300400800E052008242FCD935
:10AA1C00002000E052089B1A06D340418A42F9D12B
:10AA2C00704752089B18F8D200188A42F9D1704727
:08AA3C0010B500F071F810BD27
:10AA440038B504004D42FFF7DFFF4543611938BDB7
:10AA540070B5CC1760406140001BA141DD176A400E
:10AA64006B40521BAB4100F00BF862406340121B79
:10AA7400A3416C4060406140001BA14170BDC046D1
:10AA8400002B09D1002907D110B51100FFF7D8FF19
:10AA94000A000021002310BD70B400240125ED0735
:10AAA400002B07D1002905D0834203D213000022D2
:10AAB4002C0000250026A419994200D1904212D9F5
:10AAC40092185B4103D2EE076D086408F3E7DE07D2
:10AAD4005B08520892190126F6079B1903E0DE076A
:10AAE4005B0852089219801A994103D364416D415D
:10AAF400F5D30FE024196D410AD2DE075B08520832
:10AB0400921980185941F5D364416D41E7D301E0AE
:10AB14008018594102000B002000290070BC7047C6
:08AB2400002000217047C0462B
:10AB2C00F0B503AF93B06E46F51D2135F41D3934E5
:10AB3C0074613362F261F160306101F07CFDB060F0
:10AB4C00C21D07218A436946B1616946881A706043
:10AB5C008546F41D1D3400212422204601F050F9B5
:10AB6C000B487169F2680A6048600A4828603069CD
:10AB7C002862B06868617068E8602046F169326AE2
:10AB8C0000F01EF8B1698D46FE1F053EB546F0BDBE
:08AB9C0033C60008FFFFFF7F34
:10ABA40083B010B581B0044603A80EC00548006800
:10ABB40003AA0092214601F0B4FB01B010BC02BC10
:08ABC40003B008471400002053
:10ABCC00F0B59FB01192169106460020306001211D
:10ABDC000A020E924A020B928A020192CA02009257
:10ABEC0003220D92920205920A0317924A030692CF
:10ABFC008A0304920391C9030990C04302901496EE
:10AC0C000D460A9102E0304601F02DFB16980178B2
:10AC1C00252906D0002901D100F07BFF401C16909D
:10AC2C00F1E7C01C099E0B9C0746801E007802466B
:10AC3C00203A3E2A00D940E08021C0467A4412795D
:10AC4C0052009744233A3A203A3A3A293A3A2D2B71
:10AC5C003A1F3A3A253A3A3A3A3A3A3A3A3A3A3A78
:10AC6C003A3A3A3A3A3A3A3A3A3A3A3A3A3A3A3A38
:10AC7C003A3A3A3A3A3A3A3A3A3A3A3A3A3A3A3A28
:10AC8C003A3A270010210E43781CCDE74021FAE711
:10AC9C002146F8E71799F6E72946F4E72021F2E771
:10ACAC00119901C91191C10F09010E43C1174840F7
:10ACBC00441A3A46781E007810E07A1E0146303964
:10ACCC00002409290AD80A2161434418303C511C3C
:10ACDC0010780246303A0A2A0A46F4D300232E286A
:10ACEC000AD110782A28374609D15078921C11992C
:10ACFC0008C91191149E13E03746149E14E0521C9F
:10AD0C00014630390929149E0CD80A21594343189D
:10AD1C00303B511C10780246303A0A2A0A46F4D3CA
:10AD2C00002B01D40E990F43169201464C392E2953
:10AD3C0039D849007944898849008F442E00340061
:10AD4C003400340034003400340034003400340057
:10AD5C003400340034003400340034003400340047
:10AD6C003400340034003400340034003400340037
:10AD7C00340034003F0134002E003400390134001B
:10AD8C00340034003400340034003400300034001B
:10AD9C00340034003400340030000220074316998C
:10ADAC000878491C1691782800D92FE7E1178C43B5
:10ADBC00810001A251588F463DBB0008ADAF000881
:10ADCC00ADAF0008ADAF0008ADAF0008ADAF0008E7
:10ADDC00ADAF0008ADAF0008ADAF0008ADAF0008D7
:10ADEC00ADAF0008ADAF0008ADAF0008ADAF0008C7
:10ADFC00ADAF0008ADAF0008ADAF0008ADAF0008B7
:10AE0C00ADAF0008ADAF0008ADAF0008ADAF0008A6
:10AE1C00ADAF0008ADAF0008ADAF0008ADAF000896
:10AE2C00ADAF0008ADAF0008ADAF0008ADAF000886
:10AE3C00ADAF0008ADAF0008ADAF0008ADAF000876
:10AE4C00ADAF0008ADAF0008ADAF0008A9AF00086A
:10AE5C00ADAF0008ADAF0008ADAF0008ADAF000856
:10AE6C00ADAF0008ADAF0008ADAF0008ADAF000846
:10AE7C00ADAF0008ADAF0008ADAF0008ADAF000836
:10AE8C00ADAF0008ADAF0008ADAF0008ADAF000826
:10AE9C00ADAF0008ADAF0008ADAF0008ADAF000816
:10AEAC00ADAF0008ADAF0008ADAF0008ADAF000806
:10AEBC00ADAF0008ADAF0008ADAF0008ADAF0008F6
:10AECC00ADAF0008ADAF0008ADAF00083DB0000855
:10AEDC0089B0000835B00008ADAF0008ADAF000870
:10AEEC00ADAF0008ADAF0008ADAF0008ADAF0008C6
:10AEFC00ADAF0008ADAF0008ADAF0008ADAF0008B6
:10AF0C00ADAF0008ADAF0008ADAF0008ADAF0008A5
:10AF1C00ADAF0008ADAF000845B00008ADAF0008FC
:10AF2C00ADAF0008ADAF0008ADAF0008ADAF000885
:10AF3C00ADAF0008ADAF0008ADAF0008ADAF000875
:10AF4C00ADAF00080FB00008AFAF000841B000086B
:10AF5C008DB0000839B00008ADAF0008AFAF0008E5
:10AF6C00ADAF0008ADAF0008ADAF0008ADAF000845
:10AF7C006BB00008F3AF000831B10008ADAF0008AA
:10AF8C00ADAF000829B10008ADAF000851B1000801
:10AF9C00ADAF0008ADAF000849B00008252132E67E
:10AFAC0034E61E4604990F4300210891394626E0E9
:10AFBC00169908786C280AD1022004E016990878B2
:10AFCC00682808D1082007434878891CEAE6491C00
:10AFDC001691039902E0491C169104210F4378281D
:10AFEC0000D8E3E612E61E460E990F42394601D010
:10AFFC00D14A11403A06D217302313400893119DC1
:10B00C00AAE03D463746119E30781590641E3846AE
:10B01C002946224601F0F1FA38462F46159901F0DF
:10B02C0022F9361D119602E106980743059828E08F
:10B03C0006980743019824E006990F43BF4A7828E5
:10B04C0000D12032119D1E460E990F42394601D077
:10B05C00B94B19403B06DB17134008937CE0119A5F
:10B06C0010683907316800D55FE2BA07016001D575
:10B07C00002141601198001D1190C7E50698074307
:10B08C00009807430E98074200D106230C943946CA
:10B09C00059A1140891A4A424A41002B00D01A469F
:10B0AC001592119CE41D0720844326686568304680
:10B0BC002946FEF757FC08341194002812D00022C0
:10B0CC00304629461346FFF703FB3A4606990A40D9
:10B0DC0000280C9C17D0002A9948159B00D180E0C1
:10B0EC0098487EE030462946FEF72EFC00280C9C42
:10B0FC0000D1A7E006980742934800D093489449A2
:10B10C000F40159B6FE0002A9249159B00D0924985
:10B11C00002A62D09148BA0662D462E0119901C942
:10B12C00119160E00C9438060E990F430F97C017DD
:10B13C00232101400891119808C81190002708207C
:10B14C00079011E10E991E460F4201D07A490F402B
:10B15C003946119D0022089202220A40049B194292
:10B16C000C9406D1002A0DD12B1D00272A461D4612
:10B17C000EE0002A18D104CDD7174B071BD513B2FC
:10B18C001204A3E0EA1D07239A43576815460835B5
:10B19C0013684A071ED408220A4000D0DBB2002AEA
:10B1AC0000D19EE000279CE0ED1D0722954384CD45
:10B1BC0000354B07E3D40B0700D585E01346002F71
:10B1CC0000D486E000225C42BA412D23089323462A
:10B1DC00174686E09BB2002783E06148BA0600D58B
:10B1EC0008465B490F4000285E4E00D006460E987C
:10B1FC00074203D1304600F035FD03E030461946D6
:10B20C0000F084FD05464C480740641B14983946F1
:10B21C00224601F0F2F9002D09D00F97149F3178D6
:10B22C00384601F020F8761C6D1EF8D10F9FF806F9
:10B23C000A9D149E00D4E9E420213046224601F0F8
:10B24C00CEF9E3E430462946FEF798FB002800D1FE
:10B25C000646002800D100253046294601F069F940
:10B26C0004460120002C089001D0C00745401EAABE
:10B27C00304610952946FEF7B9FB1E980D994843A8
:10B28C000A21FFF795FB05461E90002C129601D063
:10B29C006020074300223046109C2146139213462F
:10B2AC00FFF7BCF9002800D023E1681CFEF7BEFFB5
:10B2BC0032462346FFF70CFA002800D10CE11E9809
:10B2CC00411C1E91801CF1E753B21206D71700D512
:10B2DC0078E78A0603D44A0603D5202200E02B2205
:10B2EC0008920E9A114201D0134A11400A46119548
:10B2FC000E990F920A42039900D0314607915838A3
:10B30C00002420280A9A00D997E0C0467844007996
:10B31C0040008744299292929292929292929292A7
:10B32C0047929292924792929292927C2992929206
:10B33C00924792922900C046FFFDFFFF5830000053
:10B34C0053CC00084ECC000868CE000864CE000830
:10B35C00FFFEFFFF5DCC000858CC000859CC00085C
:10B36C005ECC00086CC80008184638434DD00698CF
:10B37C000F990142F64800D0F64819093A07891886
:10B38C0000240A460F211940415C18AB19551109CC
:10B39C003F093B07C91813463B43641C002B13465B
:10B3AC00EFD14AE01846384347D00F981040109020
:10B3BC001EE015940A22002518463946139712935D
:10B3CC002B46FFF759FB04460F460A222B46FFF784
:10B3DC00D7FA2346129C201A3021014318A8159A3B
:10B3EC008154521C0920001B13988541144624D209
:10B3FC0010980028DDD020460D9908400328D8D19C
:10B40C0018A82C210155641CD3E7002415E018461C
:10B41C00384312D0D8087907401801460720184045
:10B42C00303018AA1055C808FF087A0780180A4649
:10B43C003A43641C002A0B46EFD1089DFF2D01D81E
:10B44C00029801E0C448FF300B9F0C9B07990E1B20
:10B45C00F1178E431594A1195A1A002D00D0121809
:10B46C000F99394203D1149801F0C7F800221392B6
:10B47C00290A04D0149C204600F0F5FE02E0002DB1
:10B48C00149C03D02046294600F0EDFE20460F996F
:10B49C00139A01F0B2F830212046324601F09FF8A1
:10B4AC00159F012F0ADB7D1C18A84019801E0178FE
:10B4BC00204600F0D8FE6D1E012DF5D80F98C00661
:10B4CC0026460A9D01D4FFF7A1FB20213046139A92
:10B4DC0001F085F8FFF79AFB1E98FEF7A7FE32469F
:10B4EC002346FFF7D5F8002803D01E98401E1E9067
:10B4FC00F3E73D4605980540089883021E989D4247
:10B50C00159E17D005998D4205D1864212DD042176
:10B51C00C94388420EDD01990F42109D0F9300D153
:10B52C0077E10E2838DD139E73E10170121D119224
:10B53C00FFF76CFB0E9934318842109C079506D1AD
:10B54C0012982146854A864BFEF7E4FF06E04042FE
:10B55C00FEF76CFE129A234600F0DCFD04460E4604
:10B56C0000221346FFF75AF8002813D12046314623
:10B57C00FEF7F8F9002837D0002220463146134652
:10B58C00FFF7A6F83A4606990A40002800D104E1D4
:10B59C000C9CA0E50F9759E0C143711810290E4679
:10B5AC0000DB10263A0600D533E1002900D130E14A
:10B5BC003046FEF73BFE129A2B4600F0ABFD002402
:10B5CC002246684BFEF75EFEFEF7EAFA2246664B11
:10B5DC00FEF728FA22462346FFF720F8002800D170
:10B5EC0014E1761EE4D112E10F9700222046314679
:10B5FC005D4BFFF72BF800281E9F0FD00022204632
:10B60C003146594BFEF786FF04460E460022564B38
:10B61C00FFF71CF87F1C0028F0D11E970022204653
:10B62C003146524BFFF754F800280FD00022204629
:10B63C0031464D4B00F06EFD04460E4600224B4B3E
:10B64C00FFF746F87F1E0028F0D11E970598079942
:10B65C00814202D01598014601E01598411E002840
:10B66C00139100D100210F464842FEF7DFFD029AEC
:10B67C00FEF798F922463346FEF704FE06460D46C1
:10B68C0000221092384C2346FEF7E0FF00280AD027
:10B69C001E98401C1E900022304629462346FEF779
:10B6AC0039FF06460D4612961595002F2CD00099A1
:10B6BC00084680300F9A1040884227D1102F00DBAB
:10B6CC0010273846FEF7B2FD32462B4600F022FD1D
:10B6DC00FFF79CF8024608431098139016D00C46BE
:10B6EC0010461646224A234BFFF74AF94A08C3076D
:10B6FC009A184008C90708181F49081A1F48904192
:10B70C0000D3F0E1139701E01098139080210F986B
:10B71C0006460140139A11430C98801A002901D156
:10B72C00471F00E0871F17981E9C064201D1089DF9
:10B73C004AE0032120461091FFF75AF9881C012595
:10B74C0078440079400087441B2F3B1B2F00C046D8
:10B75C0054CE000844CE0008FFFEFFFFA0C8EB85C6
:10B76C00F3CCE17F0000E03F000024400000F03FFC
:10B77C00CDCCCCCCCCCCCCCC999999999999991914
:10B78C00641E1E94002212981599ED4B00F0C2FC19
:10B79C00129015917F1E022512E0002AE7490C9C9D
:10B7AC00159B00D0B3E4B3E4A41E1E94002212989F
:10B7BC001599E44B00F0AEFC12901591BF1E109D34
:10B7CC001399C817814313917006800F00D07F1E08
:10B7DC001097204600F0FFFE632801DD781E1090C4
:10B7EC000898C0023746874312981599FFF70EF850
:10B7FC0004460E46FFF788F802460B461298159938
:10B80C00FEF724FE15901291109A75E034461E989E
:10B81C00264610387142884200DC0846FEF706FDC9
:10B82C00029AFEF7BFF8129A2B46FEF72BFD05463F
:10B83C000C461E98401CFEF7F9FC15952A4623462B
:10B84C00FEF7CAFE00281E9800D0401C0028139654
:10B85C0014D4112817D3014610391E911021081A3F
:10B86C00FEF7E4FC2A46234600F054FCFEF7CEFF1C
:10B87C0004460E4600201290159017E012940024F6
:10B88C001E94264612E000201E9028462146FEF704
:10B89C00BDFF129404460E46FFF736F802460B46DF
:10B8AC0028461299FEF7D2FD1590129138460F9941
:10B8BC008843A64900250A4608326D1C0B68496866
:10B8CC00E31A33468B411146F6D280213940139A44
:10B8DC0011434B1E0A469A41002901D00021C9434D
:10B8EC007B069B0F00D0D1431E9A891A0C9A139B8E
:10B8FC00D21A51184A1B0746D017114681430B9890
:10B90C0010300F9707420AD1012A08DB0F4620217D
:10B91C00149800F0A8FC7F1EF9D10F9A01E03A466A
:10B92C000F4640201040910603D4002809D0202156
:10B93C0004E0002801D02D2100E02B21149800F008
:10B94C0092FC0F98C0060FD4002F0DD03021149804
:10B95C0000F089FC7F1EF9D106E03020C1B21498AA
:10B96C0000F081FC002D12D06D1EE800764A1118F3
:10B97C0049681258A01A30468841EED33020A41AD8
:10B98C008E41401CA31A33468B41F8D2E6E7109740
:10B99C000F9D2C4600980440149E0BD01E98012835
:10B9AC0008DB401E1E903021304600F05CFC1E98D7
:10B9BC000028F6DC80202840139F384346D02E21E7
:10B9CC00304600F050FC102F3D463E4600DB102563
:10B9DC00E8178543002C01D1284601E01E98281A4F
:10B9EC00129CFEF723FC012E23DB159A234600F054
:10B9FC0091FBFEF70BFF04460E462F4606E0302067
:10BA0C00C1B2149800F02FFC002F12D07F1EF8004A
:10BA1C004D4A111849681258A01A30468841EED385
:10BA2C003020A41A8E41401CA31A33468B41F8D205
:10BA3C00E6E71399481B149E28460F9D06D0441A1E
:10BA4C003021304600F00FFC641CF9D301980542FC
:10BA5C0029460A9D109F30D00698014201D04521FD
:10BA6C0000E06521304600F0FEFB1E98002830D423
:10BA7C002B21304600F0F7FB1E9864280DDB642167
:10BA8C00FEF7BEFF01463031304600F0ECFB1E984D
:10BA9C006421FEF7ADFF08461E910A21FEF788FFD0
:10BAAC0001463031304600F0DEFB1E980A21FEF7CD
:10BABC009FFF3031304600F0D6FB002F01D1FFF74D
:10BACC00A5F82021304600F0CEFB7F1EF9D1FFF700
:10BADC009DF82D21304600F0C6FB1E9840421E906A
:10BAEC006428CCDAD9E7139730460A220023214682
:10BAFC00FEF7C2FF0C4607460A220023FEF7BCFFE6
:10BB0C001398401E139000D100E61A433846ECD02F
:10BB1C00FCE5F068002805D006CE083E914201D223
:10BB2C00099A4254304600F0EBFB30681FB0F0BD70
:10BB3C00304600F0E5FB02981FB0F0BD5DCC00086C
:10BB4C000000244000005940300100083801000872
:10BB5C0009490968091A4A1E9141084A1268121AC1
:10BB6C00531E9A410A4006490968081A411E884129
:10BB7C00104040427047C0461400002018000020BE
:04BB8C001C00002079
:10BB900070B5182343431848C318DD6A1846183097
:10BBA000022D10D0012D08D00024002D21D15E6A75
:10BBB0009D6AB54214D9F34315E05D6A9C6AAC42B4
:10BBC00005D9EB4306E000F0DDFB004670BDED4318
:10BBD00064191B6AE418944200D31446224606E016
:10BBE000F643AD191B6AEB18934202D3144600F0DA
:0CBBF000ACFB204670BDC046EC090020F4
:10BBFC0070B50B4616490C78002C1DD103240C6132
:10BC0C004C61144D8D61144CCC610124A4020C6266
:10BC1C0000248C624C62CC620D66104D4D66102572
:10BC2C008D660C67CC664C670D4D0F266640AE5D7D
:10BC3C000E55641C102CF8D1EFF31084012181F304
:10BC4C0010881946FFF79EFF84F3108870BDC0461C
:10BC5C00EC09002073CC0008910F002091130020F8
:04BC6C0062CC00089E
:10BC7000F0B582B0017800292FD00322014600924E
:10BC800091430D6800220192D4438607F60EB4401A
:10BC9000E4432C431E4D6719A7431E4B1F4222D17C
:10BCA00008310F1F3C6862191E46A643164217D181
:10BCB0000C6862191E46A643164214D14C686219DC
:10BCC0001E46A64316420DD18C6862191E46A64335
:10BCD00010311642E5D0083905E0002002B0F0BD71
:10BCE000394600E0091D2206019A0DD02204120EE9
:10BCF00007D02202120E06D0220E009A04D004228F
:10BD000002E0012200E002228918081A02B0F0BD08
:08BD1000FFFEFEFE8080808032
:10BD1800F0B583B0002200295DD00378002B5AD0FB
:10BD2800032302469A4300240194E4438507ED0E59
:10BD3800AC40E443156825430290044600931C4038
:10BD48006418042C2FD32748274FE9190646AE4319
:10BD58000E4228D15568211F04291ED3EE19034627
:10BD6800AB43334219D1956821460839042916D3C3
:10BD7800EB190646AE431E4211D1D56821460C394F
:10BD880004290ED3EB190646AE431E4209D1103CD6
:10BD980015691032042CD8D205E0121D02E00832D1
:10BDA80000E00C320C46280601990ED02804000E3B
:10BDB8000AD02802000E11D0280E009800D00420C6
:10BDC8000146A14203D203E00121A14200D321464A
:10BDD8000298101A4218104603B0F0BD0221A14281
:0CBDE800F5D2F5E780808080FFFEFEFEB3
:10BDF400002A03D0013A8B5C8354FBD17047C046C0
:10BE040000220B0011001A00002A02D0013A8154CA
:04BE1400FCD17047A6
:10BE1800002A09D0884207D007D2801889185242D0
:10BE28008B5C83540132FBD17047013A8B5C83549D
:04BE3800FBD1704783
:10BE3C0002480068002800D1014870471C0F002000
:04BE4C0000000020D2
:10BE50007F2805D8034A125C0348405C10407047B5
:0CBE6000002070476CCE0008DDCC00080C
:10BE6C007F2805D8034A125C0348405C1040704799
:0CBE7C00002070476CCE0008DDCC0008F0
:10BE8800000000000400000002000000080000009C
:10BE9800010000000200000004000000060000008D
:10BEA800080000000A0000000C000000100000005C
:0CBEB8002000000040000000800000009E
:10BEC400000000000000000000000000000000006E
:10BED400000000000000000000000000000000005E
:10BEE4000100000002000000030000000400000044
:10BEF4000600000007000000080000000900000020
:10BF0400000000000000000000000000000000002D
:10BF14000100000002000000030000000400000013
:0CBF24004ACA000850BF000830BF0008E7
:10BF300051BE000857C6000815C400086DBE0008B1
:10BF400063C6000823C4000847C60008E7C300080A
:10BF50004CCA0008DCCC0008DCCC0008DCCC0008B3
:10BF6000DCCC0008DCCC0008DCCC0008DCCC000811
:10BF7000DCCC0008DCCC0008FFFFFFFFFFFFFFFF69
:10BF8000FFFFFFFFFFFF000010CA00088ECC000873
:10BF900073C80008ABCC0008CAC800087CCC0008F5
:08BFA00085CC0008D1C800089F
:10BFA800034C206804348047FBE7F7F71BFDFEE7E6
:04BFB800ECCE0008C3
:10BFBC000448054988438546044880470448054998
:10BFCC000160EBE70080002007000000E7C00008DC
:08BFDC0008ED00E00000000880
:10BFE400FEE7FEE7FEE7FEE7FEE7FEE7FEE7FEE725
:10BFF400FEE7FEE7FEE7FEE7FEE7FEE7FEE7FEE715
:10C00400FEE7FEE7FEE7FEE7FEE7FEE7FEE7FEE704
:10C01400FEE7FEE7FEE7FEE7FEE7FEE7FEE7FEE7F4
:0CC02400FEE7FEE7FEE7FEE7FEE7FEE7B2
:02C03000704757
:10C0320030B580214158212918D102465632938ABF
:10C04200002B13D0016802E05B1E1C040ED0148882
:10C05200002C0CD0CC692406F6D5046D25788D62AF
:10C06200641C04651488641E1480EDE730BD012051
:10C07200C0058A6882438A600868402202430A60D7
:02C0820030BDCF
:10C0840010B5842141582229016810D102465E323C
:10C094005388496A1940836D19701188491E1180AB
:10C0A400816D491C81651188002905D010BD8869FE
:10C0B400082202438A6110BD0146843109225201DB
:10C0C40003681C6894431C609A680124A2439A6024
:0AC0D4000022C2662020086010BDA3
:02C0DE007047A9
:02C0E000FEE779
:02C0E2007047A5
:02C0E4007047A3
:02C0E6007047A1
:10C0E80008D1002806D1F54204D801D3002A01D18D
:10C0F8006D0D09D10020C143090DC904F0BDF9D166
:10C108001242F7D1640DF5D00020C1434905490812
:10C11800A6E000206146F0BDF0B50127FF070E003C
:10C128005E403E40B446BE0A4C18DD18F442D7D2F1
:10C13800F542E4D2640DECD06D0DEAD06419C90261
:10C148003943460DC0023143DB023B43DB0A10B4DE
:10C158008E4685B297B26F43140C6C433E0CA419FB
:10C16800260C2404BFB227439CB26C43A419190CB3
:10C178006943250CA4B249190D04090C6419000C73
:10C1880095B245433E0C76193743BFB2360C150CB1
:10C198004543AD19A6B2240CAD192E0437432E0C15
:10C1A80036199DB24543AD19ACB22E0C89191D0C38
:10C1B80045436D182E04290C3443704680B295B25D
:10C1C80045433E0C76193743BFB2360C150C454330
:10C1D800AD19A6B2AD19240C2E0437432E0C36190E
:10C1E8009DB24543AD19ACB22E0C89191D0C4543BF
:10C1F8006D182E043443290C75462D0C90B26843F3
:10C208003E0C80190604BFB23E43070CA0B23F188B
:10C21800120C6A43D019020C80B2240CA4189AB2EA
:10C228006A43121914042043120C89181B0C6B431F
:10C23800C91810BC01273D05294203D1B619404150
:10C248004941013CFF077D0D013D641B0BDB6D007F
:10C25800AC4209DA240500254208BE416841614123
:0AC2680066463143F0BD54E74EE78F
:10C2720030B581B06A4611700269002A17D018C819
:10C282000838A3423CD243695C1C4461D1544269E0
:10C29200002A35D081698A4232D1036A002B03D049
:10C2A20001690446984720460021416128E0C2689E
:10C2B200002A09D018C80838A34221D25D1CA54221
:10C2C20000D10021D1541BE08268002A08D018C88E
:10C2D2000838A34214D25D1CA5420ED0C9B20DE0AB
:10C2E200036A002B0CD006C80838914208D269466E
:10C2F200012204469847204602E000219B00D150CB
:0AC302000168491C016001B030BD64
:10C30C0010B54269002A07D00446036A002B01D0FD
:0AC31C00216998470020606110BD00
:10C3260070B514460D460646FFF785FD01463046B4
:0AC336002A462346FEF7F7FB70BD10
:0AC3400080B50068FFF75AFC80BDCD
:10C34A00F0B581B0154604464068A268E768C0198E
:10C35A00D61BB54204D22A46FFF747FD7D1909E0EC
:10C36A000F463246FFF741FDB919AD1B60682A46F0
:0AC37A00FFF73BFDE56001B0F0BDE8
:10C38400F0B583B016460D46C7680021019006E05B
:10C394000299C760361B2D196118002E1ED0029118
:10C3A4000269F943BA4202D95418816802E052186A
:10C3B400816854184268C91B8C4200D30C46B442AD
:10C3C40000D33446D01929462246FFF711FDE71958
:10C3D400019881688F42DBD10027D9E7084603B072
:02C3E400F0BDAA
:10C3E60010B50446002000290DD0002A0BD009788C
:10C3F60048B2002808D4002C00D021600021196022
:0EC406005960411E884110BD0120C04310BD89
:0EC41400014641391A2901D220210843704700
:0EC42200014641391A2901D2202108437047F2
:10C43000010002000400060008000A000C001000C1
:06C4400020004000800016
:10C44600806A816D40220A438265C16D04220A43D7
:04C45600C265704704
:10C45A0010B580214258212A0DD1034656331A8835
:10C46A00002A026808D0016D0C789462491C0165A3
:10C47A001888401E188010BD106888431060106824
:08C48A0040210143116010BDC7
:10C4920010B584214158222901680FD102465E322B
:10C4A20053884C6A1C40836D1C801488641E14805F
:10C4B2009B1C83651288002A05D010BD886908225A
:10C4C20002438A6110BD092252010B6893430B603B
:10C4D2008A6801239A438A600021C1668430202140
:04C4E200016010BD28
:10C4E60010B582B00B4601AC2070012120460A46E9
:10C4F60000F008F8002802D0207802B010BDC04332
:04C5060002B010BDB2
:10C50A00F0B581B01E4615460C4607461846FFF799
:10C51A0020FB0146002000290AD46543A54207D31F
:10C52A00304639462A46FFF706FF2146FEF769FAE2
:04C53A0001B0F0BD9F
:04C53E00C80F70476B
:10C54200F0B581B01C4615460091CA0017183E4648
:10C55200103EB068F1682A46FFF7E1FD0CCEFDF708
:10C5620096FE009A032A0DDB183F561E2A462346E2
:10C57200FFF7D5FD0CCF083FFDF789FE761E083F79
:10C58200012EF3D82A462346FFF7C9FD01B0F0BDBC
:10C59200F0B581B01D4616460346C800022916DBD7
:10C5A20000931F18083F4C1C304629460CCF083F09
:10C5B200FDF76DFE32462B46FFF7B1FD641E083FC4
:10C5C200022CF3D8009B083306460D4600E01B18E8
:10C5D200083B0CCB30462946FDF759FE01B0F0BDB1
:08C5E200C1174840401A7047E0
:10C5EA0070B5012A09DB0C460546561C2846214629
:0CC5FA00FFF73AFE761E012EF8D870BD47
:10C6060070B50446C80610D4880503D53025012A1E
:10C6160003DA70BD2025012A07DB561C2046294671
:0CC62600FFF724FE761E012EF8D870BD30
:10C6320010B50C46436A01212046FFF765FF10BD85
:04C6420040207047DD
:10C64600024601207F2901D9C04370471170704707
:0CC65600014661391A2900D220387047D3
:0CC66200014661391A2900D220387047C7
:0FC66E0049205265666572656E7A3D25660A0041
:0BC67D00547368756E743D25660A005A
:10C688002D2D2D204761696E204472696674204300
:07C69800414C202D2D2D0067
:0FC69F0041637475616C20543D256620430A0089
:10C6AE0041637574616C20493D2566204128776988
:10C6BE0074686F7574206761696E2074656D702083
:10C6CE00647269667420636F7272656374696F6EEB
:03C6DE00290A0026
:10C6E1004B6F7272656B74757266616B746F723DBC
:10C6F1002566205B2031202F2043656C736975739B
:03C701005D0A00CE
:10C704004552524F52204144535F313236305F53C9
:0BC7140065744461746152617465003B
:10C71F004552524F52204144535F313236305F53AE
:0BC72F00657443686F704D6F64650017
:10C73A00454550524F4D20776173206368616E679B
:10C74A00656421205765206E65656420746F2070CA
:10C75A00726573657276652063616C696272617471
:10C76A00696F6E20616E642073657474696E677395
:07C77A0020646174612100DD
:10C78100454550524F4D20464143544F5259205236
:0FC791004553544F52452F5550444154452100B4
:0FC7A0007265616420636F6E6669672E2E2E00CE
:10C7AF00666163746F727920726573746F72652E30
:03C7BF002E2E001B
:10C7C20050524F54454354494F4E3A204F425F52C4
:0BC7D20044505F4C4556454C5F320060
:10C7DD0050524F54454354494F4E3A204F425F52A9
:0BC7ED0044505F4C4556454C5F310046
:10C7F80050524F54454354494F4E3A204F425F528E
:0BC8080044505F4C4556454C5F30002B
:10C81300466C61736820756E6C6F636B2065727212
:03C823006F720031
:10C826004F5554505554535F4C56505F5348554ED0
:10C83600545F554E44455254454D5045524154550A
:03C8460052450058
:10C849004F5554505554535F4F56505F5348554EAA
:10C85900545F554E44455254454D504552415455E7
:03C8690052450035
:07C86C00286E756C6C2900B9
:10C873004A616E756172790046656272756172799B
:10C88300004D6172636800417072696C004D61799B
:10C89300004A756E65004A756C790041756775735A
:10C8A300740053657074656D626572004F63746FD5
:10C8B300626572004E6F76656D62657200446563F2
:07C8C300656D626572000063
:07C8CA00414D00504D00003C
:0FC8D1002561202562202565202554202559004A
:0EC8E00075617274206572726F72200A0D000D
:10C8EE002D2D2D204761696E202043414C202D2D8A
:02C8FE002D000B
:0AC9000054736869703D25660A0053
:10C90A002D2D2D204761696E202043414C20454E34
:06C91A0044452D2D2D0007
:0EC9200064656C746120543D256620430A0056
:0AC92E0052656620493D25660A00A7
:10C938004552524F52204144535F313236305F499D
:0EC948006E7075744D757853656C6563740080
:10C9560046697273742073746172742064657465B9
:06C966006374656421000A
:0EC96C004953454E534F523A20496E697400AC
:10C97A002E2E2E466C61736820756E6C6F636B6524
:02C98A00640047
:10C98C00466C617368206F6220756E6C6F636B20F0
:06C99C006572726F72006B
:0EC9A200466C61736820206C6F636B656400E7
:10C9B0004F5554505554535F4C56505F5348554E45
:10C9C000545F4F56455254454D504552415455526F
:02C9D000450020
:0EC9D2004F5554505554204C5650204F4B009A
:10C9E0004F5554505554535F4F56505F5348554E12
:10C9F000545F4F56455254454D504552415455523F
:02CA00004500EF
:0ECA02004F5554505554204F5650204F4B0066
:10CA100053756E646179004D6F6E64617900547571
:10CA20006573646179005765646E6573646179004C
:10CA30005468757273646179004672696461790043
:0ACA4000536174757264617900009F
:02CA4A004300A7
:02CA4C002E00BA
:10CA4E004672657175656E6379204D656173757299
:09CA5E006564203D2025640A00F6
:10CA6700492028776974686F757420636F6D7065E6
:0DCA77006E736174696F6E293D25660A00BB
:10CA84004144535F313236305F4261747465727968
:10CA940043757272656E744761696E43616C696255
:10CAA400726174696F6E53746172743A20455252A4
:10CAB4004F5220494E2043414C4942524154494F20
:10CAC4004E2C204E4F205245464552454E4345205C
:09CAD40043555252454E54210015
:10CADD004E6F726D616C207374617274207769741E
:10CAED00686F757420454550524F4D206368616ED7
:0DCAFD00676573206465746563746564008B
:10CB0A00454550524F4D2046554C4C2052455354A2
:05CB1A004F524521000F
:10CB1F00454550524F4D2053544F524520434F4E91
:05CB2F0046494721000A
:0DCB34004144533132363020496E6974009F
:10CB41002E2E2E466C617368206F6220756E6C6F9D
:05CB5100636B65640048
:10CB56002E2E2E44697361626C65206C6F636B20A8
:10CB660070726F636573732066696E697368656456
:01CB760000BE
:10CB7700466C617368204F7074696F6E6279746573
:10CB87002070726F6772616D6D206661696C656494
:01CB9700009D
:10CB98002E2E2E466C617368206C6F636B20616C5F
:0DCBA80072656164792061637469766500CF
:10CBB5002E2E2E456E61626C65206C6F636B206551
:05CBC50072726F7200A6
:10CBCA004F5554505554535F4C56505F4348495043
:10CBDA005F4F56455254454D504552415455524562
:01CBEA00004A
:10CBEB004F5554505554535F4C56505F424154541B
:10CBFB004552595F554E444552564F4C544147454B
:01CC0B000028
:10CC0C004F5554505554535F4F56505F43484950FD
:10CC1C005F554E444554454D50455241545552452F
:01CC2C000007
:10CC2D004F5554505554535F4F56505F43484950DC
:10CC3D005F4F56455254454D5045524154555245FE
:01CC4D0000E6
:05CC4E002D494E4600D7
:05CC53002D696E660072
:05CC58002B494E4600CF
:05CC5D002B696E66006A
:10CC620000000000000054545220524547474553EB
:01CC720000C1
:09CC73005465726D696E616C007C
:09CC7C00256D2F25642F25790098
:09CC850025483A254D3A255300DB
:10CC8E0053756E004D6F6E005475650057656400E8
:0DCC9E00546875004672690053617400000F
:10CCAB004A616E00466562004D6172004170720010
:10CCBB004D6179004A756E004A756C0041756700CD
:10CCCB00536570004F6374004E6F760044656300CC
:01CCDB000058
:01CCDC000057
:0DCCDD0000070320041702010857104080D3
:04CCEC00899800081B
:10CCF00056616C7565206E6F742076616C69640096
:10CD00004B6F7272656B74757266616B746F723D96
:04CD100025660A008A
:10CD14002D2D2D204761696E20447269667420436D
:0CCD2400414C20454E4445202D2D2D0093
:10CD30004552524F52204144535F313236305F5397
:10CD40006574496E7465726E616C52656665726574
:04CD50006E636500A9
:0CCD540057726974696E6720534E21000D
:10CD6000554E4B4E4F574E20434F4D4D414E440074
:10CD7000466C617368204F7074696F6E6279746578
:0CCD80002070726F6772616D6D65640059
:10CD8C00537461727420656E61626C6520726561AA
:10CD9C00646F75742070726F74656374696F6E0064
:10CDAC002E2E2E466C61736820756E6C6F636B0053
:10CDBC00466C617368204F7074696F6E627974652C
:08CDCC00206C6F636B656400CD
:10CDD4002E2E2E456E61626C65206C6F636B207025
:10CDE400726F636573732066696E69736865640046
:10CDF4004F5554505554535F4C56505F4F564552FF
:08CE040043555252454E540003
:10CE0C004F5554505554535F4F56505F4F564552E3
:08CE1C0043555252454E5400EB
:10CE24004F5554505554535F4F56505F42415454DC
:10CE34004552595F4F564552564F4C544147450051
:10CE4400303132333435363738394142434445463C
:10CE5400303132333435363738396162636465666C
:04CE64004E414E00ED
:04CE68006E616E0089
:10CE6C00202020202020202020682828282820204E
:10CE7C0020202020202020202020202020202020A6
:10CE8C00481010101010101010101010101010105E
:10CE9C0084848484848484848484101010101010FE
:10CEAC001081818181818101010101010101010157
:10CEBC00010101010101010101010110101010100B
:10CECC001082828282828202020202020202020228
:10CEDC0002020202020202020202021010101020D0
:10CEEC0061CF0008240000205D0F000061CF000816
:10CEFC00820F00200300000061CF0008860F002085
:10CF0C000300000061CF00088A0F0020030000001E
:10CF1C0061CF00088E0F00201304000073CF0008AF
:10CF2C00000000203CCF000824000000B3BF000824
:10CF3C0024BF000824BF000824BF000824BF000839
:10CF4C0024BF0008100F0020140F0020180F002021
:04CF5C000024F400B9
:10CF6000206861680834002200E042540139FCD591
:02CF7000704708
:10CF720020686168A2680C3401E08B5C8354013A3A
:04CF8200FBD5704724
:020000040801F1
:04C7FC007A463F85B5
:040000050800BFBD73
:00000001FF
